:100000000C9491010C94A3010C94A3010C947E2EEA
:100010000C94702B0C94A3010C94A3010C94A301D9
:100020000C94A3010C94A3010C94A3010C948215CD
:100030000C94A3010C94A3010C94A3010C94A301B0
:100040000C9436150C94A3010C9483340C94DD317C
:100050000C94A3010C94A3010C94A3010C94A30190
:100060000C94A3010C94A3017903140F140F8303C0
:100070008E039903A403140FA803140FB603140FDF
:10008000C003CA03D403140F140F140FE403F103C5
:10009000FE031B142114241427142C1434143C14B0
:1000A000D714D714D71449144C1455145E14D7140C
:1000B000D714D714D714D714D7146A14741480140F
:1000C00088148B1494149D14A314D714D714AC144F
:1000D000B514C014B934BB34F434F434F434F43407
:1000E000F434F434F434F434F434F434C134C33434
:1000F000C534C734C934CB34CD34CF34F434D334DD
:10010000D534D734D934DB34DD34F434DF34084A21
:10011000D73B3BCE016E84BCBFFDC12F3D6C74311B
:100120009ABD56833DDA3D00C77F11BED9E4BB4C72
:100130003E916BAAAABE000000803F05A84CCDB23C
:10014000D44EB93836A9020C50B9918688083CA61D
:10015000AAAA2ABE000000803F00536C6565706942
:100160006E6700526573746F72696E672073706991
:100170006E646C6500526573746F72696E6720649B
:10018000656661756C74730050676D20456E640020
:10019000436865636B204C696D69747300436865DF
:1001A000636B20446F6F720044697361626C6564B5
:1001B00000456E61626C65640043617574696F6EC1
:1001C0003A20556E6C6F636B656400272448277C6A
:1001D0002724582720746F20756E6C6F636B005254
:1001E0006573657420746F20636F6E74696E7565D6
:1001F000005B4D53473A000D0A4772626C20312E66
:100200003166205B27242720666F722068656C703A
:100210005D0D0A00244E005B4F50543A005B56457A
:10022000523A312E31662E32303137303330323A55
:10023000005B544C4F3A005B4739323A0033300090
:100240003238005B4700204700204D00205300203B
:10025000460020540033382E005B47433A47005B8A
:10026000484C503A24242024232024472024492089
:10027000244E2024783D76616C20244E783D6C69B4
:100280006E6520244A3D6C696E652024534C5020D5
:100290002443202458202448207E2021203F20630E
:1002A00074726C2D785D0D0A00414C41524D3A003C
:1002B0007C413A007C4F763A007C57434F3A007CB1
:1002C000506E3A007C46533A007C42663A007C57B6
:1002D000506F733A007C4D506F733A00536C6565F4
:1002E0007000446F6F723A00436865636B00416C45
:1002F00061726D00486F6D65004A6F6700486F6CF2
:10030000643A0052756E0049646C65000D0A005B2A
:100310005052423A006572726F723A006F6B0D0A6A
:10032000000011241FBECFEFD8E0DEBFCDBF27E015
:10033000A0E0B1E001C01D92A136B207E1F70E9432
:10034000B90F0C94A33A0C9400002F923F924F9255
:100350005F926F927F928F929F92AF92BF92CF9255
:10036000DF92EF92FF920F931F93CF93DF93CDB75E
:10037000DEB7CA54D1090FB6F894DEBF0FBECDBFA9
:100380008AE3E0ECF1E0DF011D928A95E9F78BE06A
:10039000E0E8F1E0A1ECB1E001900D928A95E1F77F
:1003A00080911107843211F00C94350F81E0809315
:1003B000C1011092C20183E08A8FB1E0BBA3212C5E
:1003C000312C1CA61BA610E01B8E1F8EEE24E3947E
:1003D000F12CEAE0AE2EB12CF1E68F2EF3E09F2E49
:1003E0008A8DE82FF0E0EF5EF84FD080DD2009F431
:1003F00035C29FEB9D0D9A3110F00C94040F8F5F66
:100400008A8FBE016A5E7F4FCE014A960E941F35D9
:10041000882311F40C94060F4E885F88688C798CC1
:10042000C301B2010E940E3A0E944C37062F70E0C1
:1004300080E090E00E947D379B01AC01C301B201D6
:100440000E94D33520E030E048EC52E40E942B3982
:100450000E9498390E944C37CB01E7E4DE1629F060
:10046000FDE4DF1609F4EAC033C1083209F4C6C05E
:1004700020F5043168F4013108F08AC0043009F431
:1004800052C008F464C00A3009F445C00C94140F3B
:100490000C3109F440C050F4063110F00C94140FE4
:1004A00025E1201B2093C30126E0ADC00E3199F158
:1004B000063209F44CC00C94140F0D3309F498C0A3
:1004C000A8F4053381F140F40B3209F47AC001330A
:1004D00009F477C00C94140F0C3310F00C94140F23
:1004E0006AEC600F6093C70129E08DC00C3538F4C9
:1004F0000A3508F053C0003581F10C94140F0C3507
:1005000051F00F3510F00C94140F2EE5201B2093A2
:10051000C20125E078C0009731F42F8D21110C9491
:10052000080F31E03F8F0093C001202F2D7F2C3129
:1005300019F00C3509F064C0009721F00A9711F00A
:100540000C94140F600F6093C00120E061C04F8DC8
:1005500041110C94080FA2E0AF8F0093C101063245
:1005600009F050C08431910559F08E31910541F068
:100570008832910529F08233910511F00C94140F03
:10058000B5010E94403A66576093C10121E040C026
:100590006FEE600F6093C50122E035C0892B31F406
:1005A00066EA600F6093C40123E032C06A307105CF
:1005B00011F00C94140F0A3511F40C94140F24E06C
:1005C00027C0BF8DB1110C94080F013331F4109284
:1005D000C60128E0E3E0EF8F1BC00A9711F00C94EE
:1005E000140FF1E0F093C60128E033E03F8F10C014
:1005F000892B11F00C94140F2AE00AC027E003C0E5
:1006000020E001C021E0892B19F087E10C943C0F18
:10061000C70102C0880F991F2A95E2F72BA53CA5B8
:1006200028233923232B19F085E10C943C0FABA52B
:10063000BCA5A82BB92BBCA7ABA7D2CE892B29F779
:10064000063018F4033058F016C0083010F40C943B
:10065000140F0A30F0F00E3159F00C94140F0023EF
:1006600019F0013001F104C0B3E0B093C8011BC020
:100670000093C80118C0043021F0053031F080E14A
:1006800001C080E28093CA0102C01092CA018CE0CE
:100690000BC0093021F080E48093C90102C01092A0
:1006A000C9018DE001C08BE0F70102C0EE0FFF1F12
:1006B0008A95E2F72BA53CA52E233F23232B09F097
:1006C000B3CF2BA53CA52E2B3F2B3CA72BA788CE29
:1006D0008D2DDD0C990BAA0BBB0BFC01E654F10927
:1006E000E531F10510F00C94140FEC5CFF4F0C9405
:1006F000763A4092CC015092CD016092CE01709238
:10070000CF0180E087C04092D0015092D101609229
:10071000D2017092D301116081E07CC04092D4017B
:100720005092D5016092D6017092D701126082E09A
:1007300071C04092D8015092D9016092DA01709252
:10074000DB01146083E066C00093DC0184E062C0DA
:10075000C301B2010E9445376093DD017093DE0151
:100760008093DF019093E00185E054C04092E10165
:100770005092E2016092E3017092E40186E04AC087
:100780004092E5015092E6016092E7017092E80123
:1007900087E040C04092E9015092EA016092EB018B
:1007A0007092EC0188E036C020E030E04FE753E47F
:1007B000C301B2010E94EB38181614F40C940A0F0E
:1007C0000093ED0189E026C04092EE015092EF01C6
:1007D0006092F0017092F1013B8D31603B8F8AE0B5
:1007E00019C04092F2015092F3016092F4017092AC
:1007F000F5014B8D42604B8F8BE00CC04092F601AF
:100800005092F7016092F8017092F9018B8D84602B
:100810008B8F8CE06701082E02C0CC0CDD1C0A9483
:10082000E2F7960122213321232B11F00C940C0FB7
:10083000D40102C0B595A7958A95E2F7A0FF0BC039
:1008400020E030E0A901C301B2010E94C93687FF50
:1008500002C00C940E0F2C283D28C2CDBB8DBB23AB
:1008600029F0EF8DE11102C0F2E0FF8F25FE0FC0ED
:100870008091DD019091DE01A091DF01B091E00156
:1008800081389649A849B10514F00C94100F3BA18A
:10089000332329F020FC02C00C941A0F18C0809159
:1008A000C201813071F44F8D4230E1F58091C10178
:1008B0008035C1F18823B1F120FC02C00C941A0FDD
:1008C00031C08091810181112DC020FE1BC080911B
:1008D000C301813039F523E333E34BEC51E46091FC
:1008E000CC017091CD018091CE019091CF010E94F9
:1008F0002B396093CC017093CD018093CE019093FE
:10090000CF0110C080918F0190919001A091910131
:10091000B09192018093CC019093CD01A093CE0130
:10092000B093CF0130FC10C080918B0190918C016D
:10093000A0918D01B0918E018093E9019093EA011D
:10094000A093EB01B093EC018091C001843039F4A5
:1009500026FC03C08CE10C943C0FE89426F88091AF
:10096000C501882369F0813029F48FAF1DAE92E074
:100970009BAF0BC01FAEA2E0ADAFB1E0BBAF05C0F7
:10098000E2E0EFAFF1E0FDAF1BAE8091C30181303B
:1009900021F02F8D2330C9F52FC060ECC62E61E009
:1009A000D62EE12CF12C3B8DA32EB12CC5010E2CA3
:1009B00002C0959587950A94E2F780FF12C023E361
:1009C00033E34BEC51E4D6019E966D917D918D9170
:1009D0009C91D1970E942B39F60166A777A780AB2F
:1009E00091ABFFEFEF1AFF0A24E0C20ED11C33E0F7
:1009F000E316F104D9F6CDCF8091C601813029F4F8
:100A00004B8D443011F00C94120F8CE0E4EAF1E0CD
:100A1000DE01119601900D928A95E1F78BA59CA5B8
:100A200091FD08C00091C0010A30C9F00C3509F4ED
:100A3000B3C01EC18091C701873018F08DE10C94BE
:100A40003C0F90918601891769F3BE016F5F7F4F5C
:100A50000E949B1E882311F40C94280FE3CF9B8DDA
:100A6000911103C08AE10C943C0FC1018075992754
:100A7000892B09F46FCF6091E1017091E2018091BF
:100A8000E3019091E4010E940E3A0E944C376730D6
:100A9000A8F68091DC01843141F0823011F00C9491
:100AA000140F27FE02C00C94140FAFEA2A2266230B
:100AB00019F0615069A703C0B091C701B9A760EDF3
:100AC00071E089A50E949B1E882311F40C94280FC5
:100AD0000091DC014090BC015090BD016090BE01CE
:100AE0007090BF0140ECE42E41E0F42E50E8A52EBA
:100AF00051E0B52EC12CD12CEB8D8E2E912CC40142
:100B00000C2C02C0959587950A94E2F780FF35C0BA
:100B1000043151F5D501D0962D913D914D915C91C7
:100B2000D39758966D917D918D919C915B970E9482
:100B3000D335F70126A537A540A951A90E94D33581
:100B4000D70150966D937D938D939C935397B2E00C
:100B5000CB1213C0A30192010E94D335F701608B21
:100B6000718B828B938B09C0F70186A597A5A0A9ED
:100B7000B1A9808B918BA28BB38BFFEFCF1ADF0AC9
:100B800024E0E20EF11C34E0A30EB11C43E0C416D5
:100B9000D10409F0B4CF3FC18B8D882309F462CF13
:100BA0004090BC015090BD016090BE017090BF01AB
:100BB00020E8822E21E0922EDE0111967D0130EC9C
:100BC000C32E31E0D32EA12CB12CE82FF0E0F8A7F2
:100BD000EFA38FA198A50A2C02C0959587950A943A
:100BE000E2F780FF29C0D7012D913D914D915C9195
:100BF000F401608D718D828D938D0E94D335D60165
:100C00009E962D913D914D915C91D1970E94D33547
:100C1000F60166A777A780AB91ABF2E0AF1216C0E2
:100C2000A30192010E94D335D6019E966D937D93C8
:100C30008D939C93D1970AC0F40180A991A9A2A990
:100C4000B3A9F60186A797A7A0ABB1ABFFEFAF1A88
:100C5000BF0A24E0820E911C34E0E30EF11C44E054
:100C6000C40ED11C83E0A816B10409F0B2CFD2C0E3
:100C70009F8D933069F40E3109F494C0053309F463
:100C8000C3C00C3109F0C6C060ED71E086E08DC0D4
:100C9000AB8DAA2381F3B091C401BFA34090BC01E6
:100CA0005090BD016090BE017090BF0180E8A82EF9
:100CB00081E0B82E90ECE92E91E0F92EFE013196FC
:100CC0004F01C12CD12C2A2F30E03AA729A789A5A2
:100CD0009AA50C2C02C0959587950A94E2F780FDA1
:100CE0000BC0F501808D918DA28DB38DF70186A784
:100CF00097A7A0ABB1AB44C0053309F441C0FFA135
:100D0000F1112BC0D501D0962D913D914D915C9163
:100D1000D397F40160817181828193810E94D435DF
:100D2000D7019E962D913D914D915C91D1970E9456
:100D3000D435F70166A777A780AB91ABF2E0CF126D
:100D40001FC0A30192010E94D435D7019E966D93D6
:100D50007D938D939C93D19713C0F501208D318D98
:100D6000428D538DD7019E966D917D918D919C9171
:100D7000D1970E94D435F70166A777A780AB91ABD6
:100D8000FFEFCF1ADF0A24E0A20EB11C34E0E30E1D
:100D9000F11C44E0840E911C83E0C816D10409F0D4
:100DA00096CF69CF60ED71E087E00E949B1E88239B
:100DB00011F40C94280F9B8D911103C019A61F8E5E
:100DC0002AC0A0E8B1E0E0ECF1E080E090E04B8DDB
:100DD000242F30E0A901082E02C0559547950A94AA
:100DE000E2F740FD0AC058964D915D916D917C915E
:100DF0005B97408B518B628B738B01961496349664
:100E00008330910539F706C08091C101823010F01E
:100E10000C94160F19A68091C1018FA3803529F477
:100E20009B8D91110C94180F7AC2AF8DA23009F0EE
:100E300076C2BFA1B11104C0EB8DE11170C22AC00E
:100E400020E030E0A9016091CC017091CD0180914A
:100E5000CE019091CF010E94C936882309F4EAC7D8
:100E6000FFA1FC3809F445C240F4F230A9F0F33098
:100E7000B1F0F13009F053C20AC02FA12E3809F4A5
:100E800038C208F433C22F3809F430C248C23B8D4F
:100E9000311145C21F8E43C24BA144604BA38B8DC1
:100EA000882309F4DFCDBBADAB2FB0E0B8ABAFA763
:100EB000FDADEF2FF0E0FCABEBAB81E090E07C010F
:100EC0000BAC02C0EE0CFF1C0A94E2F70DAC02C0A2
:100ED000880F991F0A94E2F7E82AF92A2B8D822FAE
:100EE00090E08E219F21892B09F4A6C7FD01EE0F0A
:100EF000FF1FEE0FFF1FE054FE4FAA0FBB1FAA0FEC
:100F0000BB1FA856BE4F2D913D914D915C9166A59A
:100F100077A580A991A90E94D3352B013C01EBA9AB
:100F2000FCA9EE0FFF1FEE0FFF1FE054FE4FABA911
:100F3000BCA9AA0FBB1FAA0FBB1FA856BE4F2D915D
:100F40003D914D915C9166A577A580A991A90E94DC
:100F5000D3354B015C01610130E8C322DD2427FE5B
:100F6000F5C0E89427F84CE050E06EEE71E088E9B7
:100F700091E00E94963A892B11F481E27DC780911D
:100F8000C3018130B1F423E333E34BEC51E46091CE
:100F9000E5017091E6018091E7019091E8010E94DE
:100FA0002B396093E5017093E6018093E7019093FC
:100FB000E8018091E5019091E601A091E701B091EF
:100FC000E8018FAB98AFA9AFBAAFA3019201C301FB
:100FD000B2010E942B3927966CAF7DAF8EAF9FAFC9
:100FE0002797A5019401C501B4010E942B392B96C6
:100FF0006CAF7DAF8EAF9FAF2B9720E030E040E825
:1010000050E46FA978AD89AD9AAD0E942B392FA914
:1010100038AD49AD5AAD0E942B3927962CAD3DAD68
:101020004EAD5FAD27970E94D3352B962CAD3DADCD
:101030004EAD5FAD2B970E94D3356B017C0120E054
:1010400030E0A9010E94C93687FDF8C6C701B60184
:101050000E94CA396B017C012B962CAD3DAD4EAD83
:101060005FAD2B9727966CAD7DAD8EAD9FAD27976D
:101070000E94D4350E94CA399B01AC01C701B60158
:1010800090580E94D3366B017C019FA1933021F4CC
:10109000F7FAF094F7F8F09420E030E0A9016FA996
:1010A00078AD89AD9AAD0E94C93687FF11C0F7FAB5
:1010B000F094F7F8F0948FA998ADA9ADBAADB058F7
:1010C0008093E5019093E601A093E701B093E801D6
:1010D0000FA518A9000F111F000F111F00531E4F5D
:1010E000A7019601C501B4010E942B399B01AC01F7
:1010F000C301B2010E94D33520E030E040E05FE35D
:101100000E942B39D8016D937D938D939C931397F7
:101110000BA91CA9000F111F000F111F00531E4F18
:10112000A7019601C301B2010E942B39A5019401C8
:101130000E94D43520E030E040E05FE30E942B398C
:10114000F8016083718382839383E9C0212F30E0AB
:1011500038AF2FABE222F322EF2809F471C631EF4A
:1011600023228091C301813009F47BC0EFA5F8A947
:10117000EE0FFF1FEE0FFF1FE053FE4FC080D18028
:10118000E280F380A7019601C301B2010E94D3352A
:101190002B013C01EBA9FCA9EE0FFF1FEE0FFF1F77
:1011A000E053FE4F80819181A281B3818FA798ABDC
:1011B000A9ABBAAB9C01AD01C501B4010E94D33506
:1011C0004B015C01A3019201C301B2010E942B39C2
:1011D0002B013C01A5019401C501B4010E942B39EA
:1011E0009B01AC01C301B2010E94D4350E94CA39EF
:1011F0004B015C01A7019601C701B6010E942B3982
:101200006B017C012FA538A949A95AA9CA01B901C6
:101210000E942B399B01AC01C701B6010E94D43555
:101220000E94CA396B017C016093E5017093E6016D
:101230008093E7019093E8019B01AC01C501B401E3
:101240000E94D3354B015C01E894B7F82AE037EDF2
:1012500043EA5BE3C501B4010E94EB3818164CF178
:101260005EC000EC11E08FA998AD0C2C02C09595E2
:1012700087950A94E2F780FF12C023E333E34BEC37
:1012800051E4D80150966D917D918D919C91539729
:101290000E942B39F801608B718B828B938BFFEF4F
:1012A000CF1ADF0A0C5F1F4F23E0C216D104D9F614
:1012B0005DCF20E030E040E05FE3C501B4010E9473
:1012C000EB3818160CF459CE2FE632E143E85AE316
:1012D000C701B6010E942B399B01AC01C501B401C5
:1012E0000E94EB3818160CF448CE19C03BA13061AF
:1012F0003BA38FA18E58823018F44BA148604BA3BA
:101300008B8D882309F4AECB4CE050E06EEE71E09B
:1013100088E991E00E94963A892B09F42ECE2BA100
:1013200021709BA190FF03C0C1018E7D03C0C1014C
:101330008E7D9C7FAF8DA111937E892B09F082C594
:101340008E01035F1F4F89E0F80111928A95E9F73A
:10135000222309F44BC08BA59CA5867B892B09F021
:1013600073C58091C001853311F081116DC58091E5
:101370008B0190918C01A0918D01B0918E01898B90
:101380009A8BAB8BBC8B9091890180918801892BC2
:101390004091CC015091CD016091CE017091CF016F
:1013A0004D875E876F87788B84608D8B809170010D
:1013B00085FF06C08EEE91E00E94E22A811146C5AB
:1013C000B8018EEE91E00E94560F80911A018111B2
:1013D00041C50E94A81C892B09F43CC580E280937A
:1013E0001A010E94BC1E0E94CA1734C58091700168
:1013F000F090890181FF26C08FA18150833018F0C1
:10140000FBA1F064FBA32B8D222339F03F8D3230FA
:1014100021F44BA140684BA315C080E1F81212C023
:101420008091800181509BA19074833030F4992386
:1014300049F09BA190629BA305C0911103C0ABA191
:10144000A062ABA38091DD019091DE01A091DF014C
:10145000B091E0018093940190939501A09396013F
:10146000B09397018091C20180938101882311F08C
:1014700088E08D8B8091CC019091CD01A091CE011F
:10148000B091CF0180938F0190939001A09391012F
:10149000B09392018D879E87AF87B88B8090E901CA
:1014A0009090EA01A090EB01B090EC01A5019401AD
:1014B00060918B0170918C0180918D0190918E01D2
:1014C0000E94C936BBA1B074EB2E811103C0EBA101
:1014D000E5FF20C0FF2071F0FBA1F7FD0BC0EE205F
:1014E00021F040E050E0BA0102C0B501A4018F2D07
:1014F0000E9408348091E9019091EA01A091EB01EA
:10150000B091EC0180938B0190938C01A0938D019D
:10151000B0938E01E1100CC080918B0190918C01F1
:10152000A0918D01B0918E01898B9A8BAB8BBC8B76
:101530008091ED01809393018091CA01909189017E
:10154000981751F049895A896B897C890E9408341F
:101550008091CA01809389019D8980918901892B9D
:101560008D8BF090C901809188018F15A9F0809131
:101570001A01823029F00E94F7338F2D0E94233206
:101580008091C901811103C01092880105C090911A
:101590008801892B809388019D8980918801892BFE
:1015A0008D8B8091C001843099F4C090E101D0907E
:1015B000E201E090E301F090E40180911A018230B1
:1015C00039F00E94F73340E0C701B6010E9495311F
:1015D0008091C501809384018091C3018093820131
:1015E0002F8D233071F58091C60180938501811183
:1015F00008C01092F6011092F7011092F8011092B3
:10160000F901C090F601D090F701E090F801F09058
:10161000F901A70196016091BC017091BD01809113
:10162000BE019091BF010E94C936882351F0C0923B
:10163000BC01D092BD01E092BE01F092BF010E94B8
:101640005C2B8091C70190918601981769F0809377
:1016500086018CE0FE013196A4EAB1E001900D9282
:101660008A95E1F70E945C2B8091C40180938301ED
:101670008091C0018632F1F138F48C3109F18E315C
:10168000F9F08A3069F04FC08C35D1F1863609F413
:1016900041C0883209F047C068E971E087E02DC099
:1016A00060ED71E089A50E94131D8091860139A526
:1016B000381339C08CE0E0EDF1E0A4EAB1E025C0D8
:1016C0008D8981608D8B4F8D442329F0B8018EEE7A
:1016D00091E00E94560FB80180ED91E00E94560FF4
:1016E0008CE0E0EDF1E0A8E9B1E001900D928A957F
:1016F000E1F719C068E971E086E00E94131D13C08C
:101700008CE0EEEEF1E0A0EBB1E001900D928A9555
:10171000E1F707C08CE0E0EBF1E0DF011D928A9574
:10172000E9F70E945C2B8091C10180938001803594
:1017300009F41CC3BF8DB23009F018C3813021F405
:10174000BE01635F7F4F06C0811109C08D89816032
:101750008D8BB8018EEE91E00E94560FFEC2825032
:10176000823008F093C28091E5019091E601A0914A
:10177000E701B091E8018F8F98A3A9A3BAA3ABADFD
:1017800094E0A99F70011124F701E856FE4FF8A7D5
:10179000EFA3970120533E4F3AA729A7D9014D90B7
:1017A0005D906D907C902081318142815381C30195
:1017B000B2010E94D4356BA77CA78DA79EA7EDAD83
:1017C000B4E0EB9F80011124980128563E4F3CAFB6
:1017D0002BAFC80180539E4F9EAF8DAFDC018D9023
:1017E0009D90AD90BC90F90120813181428153815F
:1017F000C501B4010E94D4356FA778AB89AB9AAB11
:1018000077FA709477F87094D501C401B0588B8F33
:101810009C8FAD8FBE8FF701E251FE4F2BA53CA5EB
:101820004DA55EA560817181828193810E94D3352F
:101830006B017C01F801E251FE4F2FA538A949A99F
:101840005AA960817181828193810E94D3354B01B5
:101850005C01A7019601C301B2010E942B396BAB59
:101860007CAB8DAB9EABA50194016B8D7C8D8D8D7A
:101870009E8D0E942B399B01AC016BA97CA98DA97F
:101880009EA90E94D4356BAB7CAB8DAB9EABA50102
:101890009401C301B2010E942B394B015C01A701E5
:1018A00096016B8D7C8D8D8D9E8D0E942B399B01B9
:1018B000AC01C501B4010E94D3352BA93CA94DA9A7
:1018C0005EA90E9453366B017C019BA192FF13C05D
:1018D0002DEB37E346E055EBC701B6010E94EB382C
:1018E00087FD1DC02BED3FE049EC50E4C701B60178
:1018F0000E94D33512C02DEB37E346E055E3C70114
:10190000B6010E94C936181654F02BED3FE049ECA1
:1019100050E4C701B6010E94D4356B017C01809070
:10192000640190906501A0906601B09067012F8DD1
:1019300038A149A15AA1CA01B9010E94D435A50113
:1019400094010E94D335A50194010E942B390E9475
:10195000CA394B015C0120E030E040E05FE3C701A1
:10196000B6010E942B392F8D38A149A15AA10E949E
:101970002B399F77A50194010E94D3360E94B83776
:101980000E944C377CAB6BABDB01AB2B09F4D8CEA0
:101990001D894B01A12CB12C13FF12C0C501B4014C
:1019A0000E947B379B01AC016D857E858F85988970
:1019B0000E942B396D877E878F87988B177F1D8BB1
:1019C000C501B4010E947B374B015C019B01AC0156
:1019D000C701B6010E94D3366BA37CA38DA39EA33F
:1019E000EFADB4E0EB9FC00111248C0108561E4FEF
:1019F000FC01E251FE4FD8012D913D914D915C913A
:101A000060817181828193810E94D335A501940107
:101A10000E94D33627966CAF7DAF8EAF9FAF2797CE
:101A20002BA13CA14DA15EA1CA01B9010E942B3995
:101A30009B01AC0160E070E080E090E40E94D3354F
:101A40006B017C012BEA3AEA4AE25EE36BA17CA1DE
:101A50008DA19EA10E942B394B015C0120E030E05A
:101A600040E850E4C701B6010E94D4359B01AC01A7
:101A7000C501B4010E942B396FAB78AF89AF9AAF23
:101A800020E030E040E05FE3C701B6010E942B395F
:101A900023966CAF7DAF8EAF9FAF23971F8E22240E
:101AA0002394312CEBA9FCA9E215F30509F448CEE7
:101AB000BF8DBC3008F044C02B8D3C8D4D8D5E8DAC
:101AC00023966CAD7DAD8EAD9FAD23970E942B39D3
:101AD0006B017C01A30192016FA978AD89AD9AAD2C
:101AE0000E942B39A70196010E94D4357B016C011D
:101AF000A301920123966CAD7DAD8EAD9FAD239772
:101B00000E942B394B015C012B8D3C8D4D8D5E8DE0
:101B10006FA978AD89AD9AAD0E942B399B01AC01BC
:101B2000C501B4010E94D3352B013C01EF8DEF5F5D
:101B3000EF8F470156018B8E9C8EAD8EBE8E65C099
:101B4000B10180E090E00E947B372BA13CA14DA128
:101B50005EA10E942B396B017C010E94CE366B8FF7
:101B60007C8F8D8F9E8FC701B6010E94BC394B01BF
:101B70005C01A9A5BAA5CD90DD90ED90FC90F7FA97
:101B8000F094F7F8F094ADADBEAD8D919D910D90B0
:101B9000BC91A02D8F8F98A3A9A3BAA3A7019601EA
:101BA0006B8D7C8D8D8D9E8D0E942B392B013C0180
:101BB0002F8D38A149A15AA1C501B4010E942B392A
:101BC0009B01AC01C301B2010E94D4352B013C0141
:101BD000A7019601C501B4010E942B396B017C015C
:101BE0002F8D38A149A15AA16B8D7C8D8D8D9E8D35
:101BF0000E942B399B01AC01C701B6010E94D3356D
:101C00006B8F7C8F8D8F9E8F1F8EA30192016BA592
:101C10007CA58DA59EA50E94D435EFA1F8A5608373
:101C20007183828393832B8D3C8D4D8D5E8D6FA54B
:101C300078A989A99AA90E94D435ABADBCAD6D93A2
:101C40007D938D939C93139727962CAD3DAD4EAD10
:101C50005FAD2797F80160817181828193810E9435
:101C6000D435D8016D937D938D939C931397BE01CA
:101C7000635F7F4F88E991E00E94560F80911B01BE
:101C800081116BC0BFEF2B1A3B0A0CCF8D8984608A
:101C90008D8B80911A01823009F45FC00E94F73366
:101CA00080911B01811162C0FBA1F071FF2E109287
:101CB0001F012BA123FB882780F90E94A82B86B146
:101CC000807290910001891749F084E00E94C92A2E
:101CD0000E94EB3280E00E94A82B48C0B8018EEE33
:101CE00091E00E94560F81E08093190182E00E94EA
:101CF000D92A0E94EB3280911B01811137C080915B
:101D00001A018111F6CF80911901813081F4FF20F1
:101D100051F08CE0E1E0F1E0ADE0B1E001900D9236
:101D20008A95E1F707C085E00E94C92A03C081E0D7
:101D300080931F011092190180E00E94A82B0E943D
:101D4000EB320E94552A0E94B81C0E94C4310E94A6
:101D5000542E80911F0181118CC08CE0EEEEF1E0D9
:101D6000A8E9B1E001900D928A95E1F78091C80150
:101D700080938701882309F47FC00E94F733809104
:101D8000870190911A01833041F49230D1F188E0BB
:101D90000E94D92A0E94EB3234C081E080938001F6
:101DA0001092840110928301109281011092860199
:101DB000109289011092880184E68093210180931A
:101DC000220180932301923091F064EA71E080E077
:101DD0000E949B1E8823E1F10E945C2B40E050E0B2
:101DE000BA0180E00E94BF3280E00E94233281EF7E
:101DF00091E00E94B42C88E891E00E94B42C0E94EB
:101E00004F2E109287012FC081E036C082E034C08F
:101E100088E132C086E230C089E12EC084E02CC067
:101E20008BE12AC085E228C084E126C08EE124C06F
:101E30008FE122C086E120C080E21EC082E21CC089
:101E400083E21AC084E218C080E116C08FE014C09B
:101E500087E012C08CE0EEEEF1E0A8E9B1E001907D
:101E60000D928A95E1F780E007C01A8E1BA20C94B0
:101E7000DF010E9459347ACFC65BDF4F0FB6F8946A
:101E8000DEBF0FBECDBFDF91CF911F910F91FF90AD
:101E9000EF90DF90CF90BF90AF909F908F907F900A
:101EA0006F905F904F903F902F900895FF920F9307
:101EB0001F93CF93DF938C01EB018091700185FF1D
:101EC00026C0F0901A0180E2F81629F1C8010E949C
:101ED000E22A8823E1F081E080931D0188E0F81672
:101EE00041F00E945F3482E00E94C92A0E94EB32D6
:101EF0000EC088E00E94D92A0E94EB3280911B011B
:101F0000811105C080911A018111F6CFEACF80912D
:101F10001A01823041F10E94EB3280911B01811144
:101F200022C09091DA028091D902981303C00E94D6
:101F3000D531F1CFBE01C8010E949527811113C090
:101F40008091700181FF0FC0888584FF0CC04C8197
:101F50005D816E817F8180E1DF91CF911F910F9133
:101F6000FF900C940834DF91CF911F910F91FF9057
:101F70000895CF93DF93CDB7DEB761970FB6F8948E
:101F8000DEBF0FBECDBF8091C00082608093C000D5
:101F90001092C50080E18093C4008091C1008869DF
:101FA0008093C10080E090E00E944F1E8A3009F0CB
:101FB00039C545E550E061E070E08BE291E00E94B8
:101FC000571E892B09F42EC58AB18C618AB9209AD3
:101FD0008AB1806E8AB9809181008F7E8093810062
:101FE00080918100886080938100809180008C7F47
:101FF00080938000809180008F708093800080911A
:102000006E00887F80936E0014BC15BC80916E00BA
:10201000816080936E0087B1887F87B988B18760BF
:1020200088B980916C00876080936C008091680013
:102030008260809368008CE0E1E0F1E0DF011D92B6
:102040008A95E9F7789410921A018091700184FFC3
:1020500003C081E080931A01AAE12A2EA1E03A2E62
:102060009924939480911A0191E1F10111929A952A
:10207000E9F780931A0184E680932101809322017D
:10208000809323018CE0ADE0B1E01D928A95E9F7E1
:102090001092190110921D0610921E0610921F0632
:1020A000109220068091FA018093FB0180E4E0E821
:1020B000F1E011928A95E9F764EA71E080E00E940C
:1020C0009B1E811103C087E00E94C72C0E9426340A
:1020D0003B9A43980E94C1303D98459A80E00E9407
:1020E000A82B0E94B81C0E94552A0E94C4310E944D
:1020F000593487EF91E00E94B42C8091700183FFE6
:1021000010C00E94AD2E882361F090921A0181EFD9
:1021100091E00E94B42C80E991E00E94B42C0E94CE
:102120004F2E80911A01817899F081EF91E00E9401
:10213000B42C8BEC91E00E94B42C0E944F2E909214
:102140001A0110E000E0E2E0EE2EF4E08F2E29C04C
:1021500010921A010E94DB2CF4CFE92FF0E0EF5D22
:10216000F94F80819F5F913809F490E09093FB01D3
:102170008F3FE9F08A3021F50E94EB3280911B01FC
:10218000811170CFE12FF0E0EF5EF84F1082F02F59
:10219000F170FF2E00FF18C08BE00E94C72C10E0EA
:1021A00000E09091FB018091FA019813D6CF0E9434
:1021B000D5310E94EB3280911B01882391F352CFDD
:1021C0008D3009F009C4D8CF80911107882309F414
:1021D00000C4843209F0F5C3998A809112078334D0
:1021E00009F134F4882361F0843209F006C11AC081
:1021F0008A3459F08835B1F0873409F0FEC012C036
:102200008FE592E00E94B42CDAC380911A018F7D91
:1022100009F0C5C3809113078D3309F0C8C30E942C
:10222000A501C0C3909113079111C1C3833409F470
:10223000B2C01CF4843239F0C2C3873469F08835E7
:1022400009F4C9C0BCC380911A018871F82E09F045
:10225000A6C30E943D2DB3C389E592E00E94B42C31
:10226000809180018C3838F085E592E00E94B42C92
:10227000809180018A580E948E2C86E492E00E9410
:10228000B42C809186018A5C0E948E2C86E492E0B8
:102290000E94B42C809184018F5E0E948E2C86E473
:1022A00092E00E94B42C8091820125E1281B822FAC
:1022B0000E948E2C86E492E00E94B42C80918301CF
:1022C000865A0E948E2C86E492E00E94B42C809163
:1022D00081019EE5981B892F0E948E2C8091870199
:1022E000882399F089E492E00E94B42C80918701C0
:1022F000833029F08E3139F0823039F404C080E324
:102300000E94073202C00E948E2C89E492E00E9453
:10231000B42C80918901803131F0803231F081110B
:1023200007C085E303C083E301C084E30E94073252
:1023300089E492E00E94B42C80918801882311F0F6
:1023400088E301C089E30E94073282E592E00E949F
:10235000B42C809193010E948E2C8FE492E00E9415
:10236000B42C60918F0170919001809191019091B6
:1023700092010E94572C8CE492E00E94B42C609150
:102380008B0170918C0180918D0190918E0140E0C4
:102390000E94BA2B0EC080911A01823069F40E940B
:1023A0005F3481EF91E00E94B42C88EA91E00E94B2
:1023B000B42C0E944F2E03C38111F1C2E0921A0186
:1023C00081EF91E00E94B42C81EB91E00E94B42C4B
:1023D0000E944F2E3BC080911A01813009F0EFC25C
:1023E00081EF91E00E94B42C89EB91E00E94B42C23
:1023F0000E944F2E10921A01E2C290911A0192305F
:1024000008F0CDC2893409F49DC034F4833271F0F0
:10241000883409F45AC042C1823509F4E9C08335D1
:1024200009F47EC08E3409F039C112C180911307BE
:102430008111BDC210E0BE016F5F7F4F812F0E94EE
:102440009B1E811105C087E00E94C72CF12CB7C2EA
:1024500083E492E00E94B42C163029F0173041F446
:102460008DE392E002C080E492E00E94B42C04C0AC
:1024700086E3810F0E948E2C8AE30E940732CE01F0
:1024800001960E94752C0E944F2E1F5F183099F6FE
:1024900087E392E00E94B42C80EB91E00E94752CBF
:1024A0000E944F2E81E392E00E94B42C6091BC0107
:1024B0007091BD018091BE019091BF010E94662C78
:1024C0000E944F2E0E94542E7AC28091700184FF88
:1024D00063C280921A0180911307882381F0909142
:1024E0001407911164C2893539F08A3539F088357D
:1024F00009F05DC281E003C082E001C084E00E9477
:10250000053580911B0181115AC210921A010E9457
:102510004C1580911307811152C20E94DB2C96CF7B
:10252000809113078C3409F042C2809114078035E2
:1025300009F03DC280911507811139C280E80E94DF
:10254000D92A3DC2E98A80911307811133C040E541
:1025500050E06EEA73E081E197E00E94571E892BFC
:1025600051F41092110740E550E061E177E08EEA06
:1025700093E00E94C91C8DE192E00E94B42C0E945D
:10258000882A0E944F2E87E192E00E94B42C86E5B3
:102590000E94073288E40E9407328CE20E940732D0
:1025A0008FE00E948E2C8CE20E94073280E80E940D
:1025B0008E2CFFCEA3E0A98B8D3309F0F8C183E008
:1025C000282F30E0F901EF5EF84F9081D901A25F2A
:1025D000B84F9C938F5F90819111F2CF898B40E52A
:1025E00050E061E177E08EEA93E00E94C91CE7C108
:1025F00080911307833509F0DAC18091140784357F
:1026000009F0D5C1809115078D3309F0D0C18091B3
:1026100017078111CCC180911607843239F08A32B4
:1026200039F0833209F0C3C182E003C081E001C008
:102630008FEF0E94271D81EF91E00E94B42C85E767
:1026400091E00E94B42C0E944F2E0E945F34B7C1CB
:10265000E98A8091130781111DC010E0812F0E942B
:10266000952A811104C087E00E94C72C0EC084E126
:1026700092E00E94B42C812F0E948E2C8DE30E9448
:1026800007320E94882A0E94C32C1F5F123009F46F
:1026900096C1E4CF911183C111E001C010E0BE01E9
:1026A000635F7F4FCE0141960E941F35811103C0A9
:1026B00072E0F72E84C1E98981E08E0F898BF0E00A
:1026C000EF5EF84F90819D3309F071C1112371F1D4
:1026D000482F50E0282F30E0F901EF5EF84F90814D
:1026E000241B350BD901AF5EB84F9C938F5F90814F
:1026F0009111F0CF898B0E94A501811153C16D8585
:102700007E858F8598890E940E3A0E944C37162F3D
:102710000E94F733B1E51B9FC001112440E550E052
:1027200061E177E09D5F0E94C91C90CEBE016F5FA2
:102730007F4FCE0141960E941F35882309F4B8CF00
:10274000E989F0E0EF5EF84F8081811130C1AD84FE
:10275000BE84CF84D88820E030E04FE753E4C60140
:10276000B5010E94EB3818160CF421C149805A803B
:102770006B807C80C601B5010E944C37062F20E09B
:1027800030E0A901C301B2010E94C93687FD0CC126
:10279000043608F440C0045680E0033098F510E099
:1027A000000F111F000F111F823079F0F8018330E4
:1027B00011F1813019F0E55DFE4F02C0E95CFE4F7A
:1027C0004082518262827382E4C00D5B1E4F20E022
:1027D00030E040E752E4C301B2010E942B3920E00F
:1027E00030E040E752E40E942B39F80160837183A6
:1027F00082839383CEC0E15BFE4F77FA709477F8C3
:102800007094DECF8F5F0A3008F4D1C0843009F4B1
:10281000CEC00A50C2CFC301B2010E940E3A0E943C
:102820004C3710E00132110508F0C1C0F801E75B38
:10283000FF4F0C94763A633008F4BCC060935B01A0
:10284000A8C060935E01A5C060935C0102C0609364
:102850005D010E941B159DC080917001662311F0DF
:10286000846095C08B7F93C080917001662311F0C6
:1028700080648DC08F7B8BC080917001662311F0C6
:10288000806801C08F778093700180E00E94A82B40
:1028900080C060935F017DC04092600150926101F1
:1028A000609262017092630174C040926401509220
:1028B000650160926601709267016BC08091700142
:1028C000662311F0816001C08E7F809370010E94A9
:1028D0005C2B5FC080917001662321F084FF6DC086
:1028E000806255C08F7D53C080917001662311F0C6
:1028F000886001C0877F809370010E94C13049C009
:1029000080917001662311F0806141C08F7C3FC0CF
:10291000609371013EC040927201509273016092C7
:1029200074017092750135C0409276015092770122
:1029300060927801709279012CC070E070937B01F5
:1029400060937A0126C040927C0150927D01609292
:102950007E0170927F011DC0409268015092690112
:1029600060926A0170926B0108C040926C015092B3
:102970006D0160926E0170926F010E94263409C051
:1029800080917001662311F0826001C08D7F809379
:1029900070010E94061D13C055E0F52E10C048E0DE
:1029A000F42E0DC0F82E0BC034E0F32E08C023E047
:1029B000F22E05C096E0F92E02C08AE0F82E8F2D87
:1029C00008C080911A01817211F089E0E6CB0E9463
:1029D000A5010E94D32CE3CB002329F0893209F012
:1029E000E0CB0D7FDECB813208F4DBCB8F3209F4F4
:1029F000D8CB883289F08B3389F01F3488F4212FAB
:102A000030E01F5F9FE9980FF901EF5EF84F9A31B0
:102A100008F480528083C5CB02E0C3CB04E0C1CB75
:102A200001E0BFCB87E00E94C72C8FEF0E94271DDB
:102A30000E943D2DC9CA80915C01682F20915D01E3
:102A4000422F982F917080FD94E0822F817020FD9D
:102A500080E261FD986041FD806462FD906142FD0D
:102A600080689093FC018093FD0108951F920F925E
:102A70000FB60F9211248F939F938BB19091FC010D
:102A80009C71837E892B8BB915BC9F918F910F9080
:102A90000FBE0F901F90189580916F008D7F8093CF
:102AA0006F0080918100887F816080938100109207
:102AB000FE0180915E0190911A018F3F39F42091BF
:102AC0001E06211103C0903881F402C0943069F0D1
:102AD00090E0009741F0EFE9FFE03197F1F700C097
:102AE00000000197F6CF81E001C080E09091700175
:102AF00092FF02C091E08927882311F0289A089557
:102B0000289808951F920F920FB60F9211242F93B9
:102B10003F934F935F936F937F938F939F93AF9365
:102B2000BF93EF93FF938091FE01811122C28BB17D
:102B300090910E02907E8F71892B8BB98BB1837E21
:102B400090910D02892B8BB980910C0286BD82E099
:102B500085BD81E08093FE01789480912002909160
:102B60002102892B09F0BFC08091220290914D0271
:102B7000981709F4A4C0E09122022E2F30E087E0DC
:102B8000E89FF0011124ED5DFD4FF0932102E093E9
:102B900020028281938190938900809388008081B4
:102BA000918190931C0280931B02E48180911D020D
:102BB0008E1761F1E0931D0282E1E89FF00111247C
:102BC000E25BFD4FF0931F02E0931E028485958522
:102BD000A685B785B695A7959795879580930702A3
:102BE00090930802A0930902B0930A028093030213
:102BF00090930402A0930502B09306028093FF0114
:102C000090930002A0930102B0930202A0911E02D1
:102C1000B0911F0250969C9150978091FD01892799
:102C200080930E0287E0829FF001839FF00D1124B4
:102C3000ED5DFD4F25814D915D916D917C911397D7
:102C4000022E04C076956795579547950A94D2F75A
:102C500040930F025093100260931102709312027E
:102C600014964D915D916D917C911797022E04C041
:102C700076956795579547950A94D2F74093130236
:102C800050931402609315027093160218968D915A
:102C90009D910D90BC91A02D04C0B695A7959795D8
:102CA00087952A95D2F78093170290931802A093E4
:102CB0001902B0931A0286810E94B13214C00E9498
:102CC0004C15E0911E02F0911F028189882339F092
:102CD0001092B3008091B0008F778093B00084E0B1
:102CE0000E94D92A46C1809119018130B1F486B180
:102CF000807290910001891781F0109219018CE087
:102D0000E1E0F1E0ADE0B1E001900D928A95E1F7EC
:102D100080911D06806480931D0610920D024091E3
:102D2000FF015091000260910102709102028091B6
:102D30000F0290911002A0911102B0911202840F23
:102D4000951FA61FB71F8093FF0190930002A093C9
:102D50000102B0930202E0911E02F0911F0244852D
:102D6000558566857785481759076A077B0768F593
:102D700024E020930D024485558566857785841B64
:102D8000950BA60BB70B8093FF0190930002A093C5
:102D90000102B09302022089809101019091020109
:102DA000A0910301B091040125FF04C00197A1097E
:102DB000B10903C00196A11DB11D8093010190933B
:102DC0000201A0930301B0930401409103025091CA
:102DD00004026091050270910602809113029091A5
:102DE0001402A0911502B0911602840F951FA61F20
:102DF000B71F8093030290930402A0930502B0933F
:102E000006024485558566857785481759076A0700
:102E10007B0778F520910D02286020930D024485F0
:102E2000558566857785841B950BA60BB70B80931C
:102E3000030290930402A0930502B0930602208936
:102E40008091050190910601A0910701B0910801C0
:102E500026FF04C00197A109B10903C00196A11D75
:102E6000B11D8093050190930601A0930701B093D3
:102E70000801409107025091080260910902709187
:102E80000A028091170290911802A0911902B09144
:102E90001A02840F951FA61FB71F809307029093F5
:102EA0000802A0930902B0930A02448555856685FD
:102EB0007785481759076A077B0778F520910D0237
:102EC000206120930D024485558566857785841B96
:102ED000950BA60BB70B8093070290930802A09363
:102EE0000902B0930A0220898091090190910A0198
:102EF000A0910B01B0910C0127FF04C00197A1091B
:102F0000B10903C00196A11DB11D809309019093E1
:102F10000A01A0930B01B0930C0180911A01843037
:102F200039F490910D0280912001892380930D0244
:102F300080911B0290911C02019790931C02809338
:102F40001B02892B69F410922102109220028091B9
:102F500022028F5F80932202863011F410922202A7
:102F600090910D028091FC01892780930D021092AF
:102F7000FE01FF91EF91BF91AF919F918F917F9152
:102F80006F915F914F913F912F910F900FBE0F90D6
:102F90001F9018958091700182FF02C0289A01C08D
:102FA00028988091FC0180930D0280915B01880F2D
:102FB0008450819580930C0280916F008260809391
:102FC0006F0008953F924F925F926F927F928F921F
:102FD0009F92AF92BF92CF92DF92EF92FF920F93A8
:102FE0001F93CF93DF93CDB7DEB7A4970FB6F894B6
:102FF000DEBF0FBECDBF10911E06112391F181E0FF
:1030000080931A0189EA92E00E94B42C812F0E94D9
:103010008E2C0E94C32C85EF91E0019739F0EFE9E7
:10302000FFE03197F1F700C00000F7CF11501230E8
:1030300030F08FB7F89410921E068FBF12C081EF48
:1030400091E00E94B42C8FED91E00E94B42C0E947C
:103050004F2E80E10E94CF2A80911D0684FFFCCF75
:10306000E8CF10911D06112309F4BBC214FF04C060
:1030700081E080931B01BFC310FFBFC18CE0E1E082
:10308000F1E0DE01599601900D928A95E1F7BE01BB
:10309000675E7F4FCE010D960E94202B8CE30E942D
:1030A000073280911A018830E1F058F4813099F1AB
:1030B000A8F0823099F1843009F043C084EF92E0A7
:1030C0003EC0803229F118F4803171F03AC080346A
:1030D00041F18038B1F58CED92E031C087E093E0AA
:1030E0002EC083E093E02BC080911C0187FD10C0AF
:1030F0008DEF92E00E94B42C80911C0180FF06C0ED
:1031000080E31AC082FF17C085FFFACF81E314C0A5
:1031100089EF92E014C08EEE92E011C088EE92E04A
:103120000EC082EE92E00E94B42C80911C0183FFBD
:10313000E9CF83E301C082E30E94073202C00E940C
:10314000B42C80915F01F82FF170BF2E80FF07C073
:1031500080912601882319F085ED92E053C04090BC
:10316000BC015090BD016090BE017090BF0144EA67
:10317000842E41E0942E9E012F5F3F4F7901CE01B6
:103180000D966C0100E0F401619171918191919132
:103190004F0120853185428553850E94D435F70142
:1031A0006083718382839383023061F4A30192016F
:1031B0000E94D435F7016083718382839383BB209F
:1031C00019F0CACFB11011C0F701208131814281BD
:1031D0005381F60160817181828193810E94D33590
:1031E000F60160837183828393830F5FF4E0EF0EB7
:1031F000F11C24E0C20ED11C033029F6B110ACCF73
:103200008EEC92E00E94B42CCE010D960E94752C9B
:1032100080915F0181FF1FC089EC92E00E94B42C75
:103220009091FB058091DA02981710F0815F01C040
:103230008150891B0E948E2C8CE20E940732809163
:10324000FB019091FA01981710F0805801C081504D
:10325000891B0E948E2C84EC92E00E94B42C8091F9
:103260001A018C7749F06091BF027091C002809181
:10327000C1029091C20203C060E070E0CB010E94E5
:10328000572C8CE20E94073260912701709128012F
:103290008091290190912A0140E00E94BA2B0E945E
:1032A000AD2EF82E0E94612B082F86B1982F9072B8
:1032B00080910001E92EE8268F2D802B8E2959F16F
:1032C0008FEB92E00E94B42CEE2019F080E50E9472
:1032D0000732FF2079F0F0FE03C088E50E94073234
:1032E000F1FE03C089E50E940732F2FE03C08AE5C1
:1032F0000E940732002379F000FF03C082E50E949C
:10330000073201FF03C088E40E94073202FF03C0B6
:1033100083E50E94073280912601882321F08150A5
:103320008093260118C080911A018C7711F08DE1ED
:1033300001C089E08093260180912501811103C09D
:1033400081E08093250189EB92E00E94B42CCE01AC
:1033500001960E94752C00912501002321F0015057
:103360000093250142C080911A018C7711F083E10E
:1033700001C089E08093250184EB92E00E94B42C87
:10338000809121010E948E2C8CE20E940732809154
:1033900022010E948E2C8CE20E9407328091230130
:1033A0000E948E2C8091B00087FF05C02D9B02C02B
:1033B00002E001C001E0439B03C0FF24F39403C07B
:1033C000002399F0F12C80EB92E00E94B42C0023B2
:1033D00039F0013011F483E501C083E40E94073223
:1033E000FF2019F086E40E9407328EE30E94073224
:1033F0000E94C32C81E00E94CF2A812F887E09F48D
:1034000067C080911A01982F937009F050C088729C
:10341000A1F080911C01807C81F40E94292682E029
:1034200080931E0180911A01803239F417FDE1C1A9
:1034300080911C01806880931C0180911A01811188
:1034400003C091E090931C0116FF07C085FD05C0E5
:1034500090911C01906490931C0113FF05C0807E25
:1034600019F480E180931A0115FF21C081EF91E0EA
:103470000E94B42C8DE991E00E94B42C0E944F2E42
:1034800080911C0187FD0EC090911A01903439F48F
:1034900083FFABC1837E826080931C01A6C19038FC
:1034A00009F0A3C180911C01806280931C0117FF69
:1034B0000CC080911A01813029F480911C01856033
:1034C00080931C0180E880931A0188EE0E94CF2A25
:1034D00011FF44C0812F8876F1F580911A01803464
:1034E00071F480911C0185FD0AC084FF03C0109215
:1034F0001A0105C082FF03C0886080931C0180917F
:103500001A01882381F084FF26C090911C0190FF4E
:1035100022C0803141F480912401882321F0886009
:103520008093240118C010921E010E94A81C892BB0
:1035300071F080911C0186FD0AC010921C0188E088
:1035400080931A010E94BC1E0E94CA1704C01092E8
:103550001C0110921A0182E00E94CF2A12FF41C082
:1035600080911A01807D90911C018823D9F080916F
:103570001D01811117C097FD15C00E942926809159
:10358000DA028093D8020E944D2680911E0181FFAD
:1035900005C090911C01916090931C01897F8093DC
:1035A0001E011CC097FF0AC010921E010E94B81C89
:1035B0000E94552A0E9459340E94C43180911C01F6
:1035C00085FF08C08F77816080931C0180E4809321
:1035D0001A0104C010921C0110921A0184E00E948A
:1035E000CF2A90911F06992309F4ABC08FB7F894A6
:1035F00010921F068FBF4091210190FD02C0842FC1
:1036000001C084E691FD865F92FD8A5093FD8F5F35
:1036100094FD8150893C08F088EC8A3008F48AE0F7
:103620003091220195FD02C0232F01C024E696FDB2
:1036300022E397FD29E1481303C0231709F481C051
:103640008093210120932201109225011091DA022A
:103650003090FB0589E9D82E96E7E92E26E9F22E6F
:103660000EE732E3432E131509F457C0812E912C37
:10367000489CC001499C900D1124FC01E552FD4F6E
:103680005F01CF010E94351C562E672E782EC92E61
:103690002D2D3E2D4F2D502F0E94EB3818164CF437
:1036A0002D2D3E2D4F2D502F6D2D7E2D8F2D902F9A
:1036B00008C0252D362D472D5C2D652D762D872DA7
:1036C0009C2D0E942B39F501668B778B808F918F13
:1036D000489CC001499C900D11249C0125523D4FEE
:1036E0007901F90182A093A0A4A0B5A0A50194013D
:1036F00066897789808D918D0E94EB3818162CF49D
:10370000F701868A978AA08EB18E1F5F103109F467
:1037100010E0D52C73010C2DA6CF8D2D9E2DAF2D35
:10372000B02F8093190690931A06A0931B06B093AE
:103730001C060E9429268091DA028093D8020E94FA
:103740004D2690912006992309F448C08FB7F8942C
:10375000109220068FBF2091230190FD02C0822F7E
:1037600001C084E691FD865F92FD8A5093FD8F5FD4
:1037700094FD8150893C08F088EC8A3008F48AE096
:10378000281749F020911E01286020931E01809384
:1037900023011092250180911A0195FF0DC08031FF
:1037A00059F420912401211102C022E003C020FF1E
:1037B00003C0246020932401907C81F0882311F0C1
:1037C000887161F01091880116FF02C01F7B01C053
:1037D0001064812F0E9423321093880180911A0176
:1037E0008C7F49F00E94BC1E06C080E480931A01C1
:1037F00059CE80E229CEA4960FB6F894DEBF0FBE54
:10380000CDBFDF91CF911F910F91FF90EF90DF908F
:10381000CF90BF90AF909F908F907F906F905F9070
:103820004F903F900895F894F999FECF92BD81BDD5
:1038300081E08FBB80B58627482F082E000C550BE2
:10384000262F30E024233523232B39F06F3F19F046
:1038500060BD84E006C084E104C0882321F060BD1F
:1038600084E28FBBF99A78940895BF92CF92DF9249
:10387000EF92FF920F931F93CF93DF937C01FC0194
:1038800002A513A5D4A5C5A5818980FF18C06091A4
:10389000220170E080E090E00E947D372AE037ED61
:1038A00043E25CE30E942B399B01AC01B8018D2FF0
:1038B0009C2F0E942B398B01D82FC92F2DC082FD40
:1038C00017C06091210170E080E090E00E947D3798
:1038D0002AE037ED43E25CE30E942B399B01AC0107
:1038E000B8018D2F9C2F0E942B398B01D82FC92F07
:1038F000F701B6A0C7A0D0A4F1A42B2D3C2D4D2DCF
:103900005F2DB8018D2F9C2F0E94EB38181624F4E0
:103910000B2D1C2DDD2DCF2D20E030E040E85FE3A6
:10392000B8018D2F9C2F0E94EB38181624F000E070
:1039300010E0D0E8CFE3B8018D2F9C2FDF91CF911D
:103940001F910F91FF90EF90DF90CF90BF9008955F
:103950008091DA029091FB05981739F022E3829F5B
:10396000C001112485529D4F089580E090E0089594
:103970008CE1E1E0F6E0DF011D928A95E9F7109213
:10398000DA021092FB0581E08093D9021092D802EE
:1039900008959F92AF92BF92CF92DF92EF92FF92E3
:1039A0000F931F93CF93DF935C018A017B01E40E99
:1039B000F51EEB01912C6C01C61AD70ACE018C0DB5
:1039C0009D1DCE15DF0589F0911008C0292D990C99
:1039D000330B232F221F2227221F01C021E06991D0
:1039E000922E960E0E94131CE9CF692DC501800FFF
:1039F000911FDF91CF911F910F91FF90EF90DF907A
:103A0000CF90BF90AF909F900C94131C6AE080E021
:103A100090E00E94131C45E550E06BE271E081E00C
:103A200090E00C94C91C0F931F93CF93C82F8B0168
:103A30000E94F7332DE0C29FC00111244CE050E0FA
:103A4000B8019E5FCF911F910F910C94C91CEF920A
:103A5000FF920F931F93CF93DF93CDB7DEB72C97D1
:103A60000FB6F894DEBF0FBECDBF182F80FFD6C0B3
:103A70008AE080935B018FEF80935E0110925C017E
:103A800010925D0181E080935F018AE097EDA3E2EF
:103A9000BCE38093600190936101A0936201B093B5
:103AA00063018FE692E1A3E0BBE38093640190930E
:103AB0006501A0936601B093670180E090E0AAE7FA
:103AC000B4E48093680190936901A0936A01B09374
:103AD0006B0110926C0110926D0110926E011092A8
:103AE0006F011092710180E090E0A8ECB1E4809346
:103AF000720190937301A0937401B093750180E0FB
:103B000090E0AAEFB3E48093760190937701A093BD
:103B10007801B09379012AEF30E030937B01209354
:103B20007A0140E050E060E87FE340937C015093ED
:103B30007D0160937E0170937F0124E020937001EA
:103B400040E050E06AE773E440932B0150932C016E
:103B500060932D0170932E0140932F0150933001FB
:103B600060933101709332014093330150933401DB
:103B7000609335017093360180933701909338013B
:103B8000A0933901B0933A0180933B0190933C019B
:103B9000A0933D01B0933E0180933F01909340017B
:103BA000A0934101B093420180E090EAACE0B7E419
:103BB0008093430190934401A0934501B093460143
:103BC0008093470190934801A0934901B0934A0123
:103BD00080934B0190934C01A0934D01B0934E0103
:103BE00080E090E0A8E4B3EC80934F019093500103
:103BF000A0935101B09352018093530190935401CB
:103C0000A0935501B09356018093570190935801AA
:103C1000A0935901B0935A010E94061D11FF10C0D4
:103C2000CE0101967C018CE0F70111928A95E9F7AB
:103C300000E0B701802F0E94131D0F5F0830C9F705
:103C400012FF14C060E080E093E00E94131C60E06B
:103C500081E093E00E94131C60E081E593E00E9404
:103C6000131C60E082E593E00E94131C13FF0AC05E
:103C700060E08EEA93E00E94131C60E08FEA93E01C
:103C80000E94131C2C960FB6F894DEBF0FBECDBF5A
:103C9000DF91CF911F910F91FF90EF900895F999C7
:103CA000FECF92BD81BD81E08FBB80B508959F920C
:103CB000AF92BF92CF92DF92EF92FF920F931F933A
:103CC000CF93DF935B018A017C01E40EF51EEC01CA
:103CD000912C6B01C81AD90AC6018C0F9D1FCE15F5
:103CE000DF0589F00E944F1E911008C0292D990C04
:103CF000330B232F221F2227221F01C021E0982EE1
:103D0000920E8993E9CFC501800F911F0E944F1E2B
:103D100021E030E0981611F020E030E0C901DF9199
:103D2000CF911F910F91FF90EF90DF90CF90BF90B8
:103D3000AF909F9008951F93CF93DF93182FEB01BF
:103D40008DE0189FB00111247E5F4CE050E0CE0161
:103D50000E94571E892B59F48CE0FE0111928A951E
:103D6000E9F7BE01812F0E94131D80E001C081E0B0
:103D7000DF91CF911F9108952F923F924F925F92C2
:103D80006F927F928F929F92AF92BF92CF92DF926B
:103D9000EF92FF920F931F93CF93DF93CDB7DEB7D0
:103DA000EF970FB6F894DEBF0FBECDBF80911E0116
:103DB00080FD36C7909122028091FC05981709F486
:103DC0002FC78091FF0590910006892B09F015C33C
:103DD00010911E0112FF09C08091FB0522E3289F6C
:103DE000C001112485529D4F02C00E94A81C9093CF
:103DF00000068093FF052090FF05309000062114F7
:103E0000310409F40DC70091A902802F817000FFD1
:103E100003C01092A902EAC09091A8029F5F95305A
:103E200009F0892F8093A802E82EF12C32E13E9D03
:103E3000F0013F9DF00D1124E25BFD4FF093FE0574
:103E4000E093FD05D10150969C915097908BE2E153
:103E50008E9FC001112420E030E04D915D916D9165
:103E60007D91F901E80FF91FE25BFD4F689412F8AC
:103E7000440F551F661F771F1694D1F74083518357
:103E8000628373832C5F3F4F2C30310531F722E181
:103E90002E9DF0012F9DF00D11249F01225B3D4FBF
:103EA000F10184859585A685B78543E0880F991F24
:103EB000AA1FBB1F4A95D1F7F90184879587A6876A
:103EC000B787D1011C966D917D918D919C911F9723
:103ED0000E947B376093AE027093AF028093B00272
:103EE0009093B102F101268D378D40A151A10E941E
:103EF000D3369B01AC016093B2027093B3028093FE
:103F0000B4029093B50260E070E080EA9FE30E9403
:103F1000D3366093B6027093B7028093B802909341
:103F2000B9021092AA021092AB021092AC02109247
:103F3000AD0211FD02C003FF1FC06091C702709166
:103F4000C8028091C9029091CA026093BF02709327
:103F5000C0028093C1029093C2029B01AC010E94F7
:103F60002B39D10152966D937D938D939C935597E8
:103F7000077F0093A9020FC0F101628973898489C8
:103F800095890E94CA396093BF027093C0028093E2
:103F9000C1029093C202F2E1FE9DC001FF9D900D0F
:103FA00011249C01225B3D4F7901D90151961C924D
:103FB0008091700181FF1AC0F101818985FF16C0CF
:103FC00022A533A544A555A560E070E080E89FE3F5
:103FD0000E94D3366093D3027093D4028093D502AB
:103FE0009093D602E1E0D7015196EC931092BB0278
:103FF0001092BC021092BD021092BE02D1015A96DC
:104000002D913D914D915C915D972D833E834F8322
:10401000588760E070E080E09FE30E94D3364B0158
:104020005C01F101468C578C60A071A011FF4BC060
:10403000F2E0F093BA02D1015296CD90DD90ED906E
:10404000FC905597A70196010E942B399B01AC016A
:10405000C301B2010E94D3354B015C0120E030E086
:10406000A9010E94C93687FF1DC02D813E814F8165
:104070005885CA01B9010E94D435A30192010E945A
:104080002B399B01AC01C701B6010E94D3350E94B8
:10409000CA396093C7027093C8028093C902909393
:1040A000CA02A8C18092BB029092BC02A092BD023B
:1040B000B092BE021092C7021092C8021092C902BA
:1040C0001092CA0297C11092BA024092CB0250924B
:1040D000CC026092CD027092CE0212FF0CC0109200
:1040E000C7021092C8021092C9021092CA02C12CD3
:1040F000D12C760124C0E091DA02EF5FE03109F4BF
:10410000E0E08091FB058E1759F0B2E3BE9FF0010D
:104110001124E552FD4FC288D388E488F58803C096
:10412000C12CD12C7601C701B6010E94CA39609317
:10413000C7027093C8028093C9029093CA02C1015A
:104140000E94351C698B7A8B8B8B9C8B9B01AC01FD
:104150000E942B3969877A878B879C87D101529679
:104160002D913D914D915C91559729833A834B83D5
:104170005C830E94C93687FF6CC029853A854B85D0
:104180005C8569817A818B819C810E94D335A501F0
:1041900094010E942B399B01AC01C301B2010E9422
:1041A000D3356093CB027093CC028093CD02909371
:1041B000CE0220E030E0A9010E94C93618163CF179
:1041C000B2E0B093BA022D813E814F815885CA0179
:1041D000B9010E94D435A30192010E942B399B01A1
:1041E000AC0169817A818B819C810E94D3350E94C8
:1041F000CA396093C7027093C8028093C902909332
:10420000CA028091A90288608093A902F3C0A70125
:10421000960169857A858B859C850E94D335A50199
:1042200094010E942B396093CF027093D002809347
:10423000D1029093D20229893A894B895C892093D3
:10424000C3023093C4024093C5025093C60233E0C8
:10425000B6C0A701960169817A818B819C810E94F9
:10426000D335A50194010E942B39A30192010E942C
:10427000D43520E030E040E05FE30E942B396D87C9
:104280007E878F87988B20E030E0A9010E94EB3871
:1042900018160CF097C02D853E854F855889C301AF
:1042A000B2010E94EB3818160CF088C0A7019601E5
:1042B00069857A858B859C850E94D335A5019401FB
:1042C0000E942B399B01AC016093CF027093D00206
:1042D0008093D1029093D2026D857E858F859889D7
:1042E0000E94EB381816CCF589899A89AB89BC896C
:1042F0008093C3029093C402A093C502B093C602F8
:1043000029813A814B815C8169857A858B859C8581
:104310000E94C936811104C091E09093BA026AC02C
:1043200029813A814B815C8169857A858B859C8561
:104330000E94D335A50194010E942B399B01AC0149
:10434000C301B2010E94D3356093CB027093CC02BB
:104350008093CD029093CE024DC02D853E854F8532
:1043600058892093CB023093CC024093CD025093D6
:10437000CE022093CF023093D0024093D1025093CB
:10438000D2022D813E814F815885CA01B9010E9418
:10439000D4352D853E854F8558890E942B39A7013C
:1043A00096010E94D4350E94CA396093C30270936B
:1043B000C4028093C5029093C6021CC032E03093C1
:1043C000BA0218C01092CB021092CC021092CD0209
:1043D0001092CE028091C7029091C802A091C902AA
:1043E000B091CA028093C3029093C402A093C50205
:1043F000B093C602186010931E0180914D02482FA1
:1044000050E05E834D8387E0849FF001859FF00D2F
:104410001124ED5DFD4F8091A8028483A091FF05DA
:10442000B0910006BFAFAEAF5E96BC91BEA3EEAD3D
:10443000FFADF78DFFA3AEADBFAD9096BC91B8A711
:10444000EEADFFADF1A1F9A72091B6023091B70210
:104450004091B8025091B9026EA17FA18B2F9F2F7E
:104460000E94D3356AAB7BAB8CAB9DAB20E030E0D8
:10447000A9010E94C93687FF04C01AAA1BAA1CAA58
:104480001DAA2091CB0229873091CC023D87409113
:10449000CD02498B5091CE025D8B8091C3028A8FF1
:1044A0009091C4029B8FA091C502AC8FB091C602BF
:1044B000BD8F6090BF027090C0024090C1025090CA
:1044C000C202E091CF02EAA7F091D002FBA72091AF
:1044D000D1022CA73091D2023DA74091BA02498364
:1044E0005091BB025EA78091BC028FA79091BD0244
:1044F00098ABA091BE02A9ABB091C702BFABE0914F
:10450000C802E8AFF091C902F9AF2091CA022AAF00
:104510002AA53BA54CA55DA569857D8589899D89D1
:104520000E94C936811103C032E03EAB02C041E0B7
:104530004EAB2EA03FA008A519A58EE3C82E83EC94
:10454000D82E8EE2E82E89E3F82E1E8A1F8A188E56
:10455000198ECE8EDF8EE8A2F9A29981913009F4EE
:10456000D4C008F472C0AEADBFAD5A962D913D9146
:104570004D915C915D97933009F0F9C0C701B60188
:104580000E942B394B015C0120E030E040E05FE30A
:104590000E942B399B01AC01B301C2010E94D335AB
:1045A000A70196010E942B396AA37BA38CA39DA32C
:1045B0009B01AC01B101C8010E94D3351B018C01E4
:1045C00029853D8549895D890E94C93687FD0BC0D3
:1045D00020E030E0A9016AA17BA18CA19DA10E94ED
:1045E000C93618165CF129853D8549895D896EA11A
:1045F0007FA188A599A50E94D3359B01AC010E949B
:10460000D4356B017C019301A2016A8D7B8D8C8D69
:104610009D8D0E94D4359B01AC01C701B6010E945B
:10462000D3366B017C016A8C7B8C4C8C5D8C29842D
:104630003D8409891D89B1E0B983FFC0A5019401BA
:10464000B301C2010E94D3355DC0EEADFFAD228D36
:10465000338D448D558DC701B6010E942B394B0116
:104660005C0120E030E040E05FE30E942B399301E1
:10467000A2010E94D435A70196010E942B399B010B
:10468000AC01B101C8010E94D3351B018C019B0113
:10469000AC0169857D8589899D890E94EB38181652
:1046A0005CF529853D8549895D896EA17FA188A535
:1046B00099A50E94D3359B01AC010E94D4356B01B2
:1046C0007C019301A2016A8D7B8D8C8D9D8D0E9452
:1046D000D4359B01AC01C701B6010E94D3366B01F2
:1046E0007C016A8C7B8C4C8C5D8CFEA9F9832984BF
:1046F0003D8409891D89A1C0A5019401B301C201AE
:104700000E94D4353B012C0198C02A8D3B8D4C8DE5
:104710005D8DC701B6010E942B399B01AC01B1012F
:10472000C8010E94D3355B014C019B01AC016AA515
:104730007BA58CA59DA50E94EB3818160CF07BC0BC
:104740002AA53BA54CA55DA5B101C8010E94D335A2
:104750002A8D3B8D4C8D5D8D0E94D3366B017C0183
:104760002AA43BA40CA51DA522E0298366C0C7018D
:10477000B6010E942B394B015C019301A2010E94FA
:10478000C93687FF31C020E030E040E05FE3C5017B
:10479000B4010E942B399B01AC01B301C2010E94FC
:1047A000D335A70196010E942B399B01AC01B101C1
:1047B000C8010E94D3356AA37BAF8CAF9DAF2EA5F5
:1047C0003FA548A959A90E94EB3818166CF4A50119
:1047D0009401B301C2010E94D3353B012C012AA0F0
:1047E0003BAC0CAD1DAD29C02EA53FA548A959A9CC
:1047F000B101C8010E94D3359B01AC010E94D435A0
:104800006B017C019301A2016FA978AD89AD9AADCE
:104810000E94D4359B01AC01C701B6010E94D3367A
:104820006B017C016FA878AC49AC5AAC2EA43FA4B4
:1048300008A919A902C015018401A70196016E8972
:104840007F89888D998D0E94D4356E8B7F8B888F60
:10485000998F2E8D3F8D48A159A10E94C93687FF9F
:1048600009C02E893F89488D598D6E8D7F8D88A115
:1048700099A11CC02AA93BA94CA95DA9B101C801F5
:104880000E94EB38181624F52EE333EC4EE259E380
:104890006E8D7F8D88A199A10E94D4356E8F7F8FF8
:1048A00088A399A32E893F89488D598D0E94D335BD
:1048B0006B017C019101A8016EA57FA588A999A92A
:1048C0000E94C93687FD49CEB981B093BA0203C0B0
:1048D000E981E093BA02C301D2018093BF029093B1
:1048E000C002A093C102B093C202E091FD05F09115
:1048F000FE059189911104C080911E0183FF3FC084
:10490000AEADBFAD51968C915197807349F19E9693
:10491000CD90DD90ED90FC90D1979923D1F020912E
:10492000D3023091D4024091D5025091D6026091C9
:10493000BF027091C0028091C1029091C2020E9498
:104940002B399B01AC01C701B6010E942B396B01C9
:104950007C01C701B6010E9430328093D7020AC0A1
:1049600010922701109228011092290110922A0119
:104970001092D70280911E01877F80931E0147E02D
:104980002D813E81429FF001439FF00D1124ED5D8A
:10499000FD4FFA87E9878091D70286832091B20282
:1049A0003091B3024091B4025091B502B101C801F7
:1049B0000E942B392B013C010E94B2366B017C0115
:1049C0006091AE027091AF028091B0029091B102FD
:1049D0000E94B2364B015C01A70196010E94D335BB
:1049E0000E944C3769837A838B839C83E981FA81A7
:1049F000A985BA85ED93FC93EF2B41F480911E01BC
:104A000081FF04C0816080931E010AC12091AA0227
:104A10003091AB024091AC025091AD026E897F891A
:104A2000888D998D0E94D43569877A878B879C877A
:104A3000A3019201C501B4010E94D3359B01AC01D1
:104A400069857A858B859C850E94D3364B015C01F4
:104A500020EC31EE44E65EE40E942B390E94B2362F
:104A60000E944C37603D37E073078105910560F483
:104A7000A7E04D815E81A49FF001A59FF00D112458
:104A8000ED5DFD4F158253C0603ABFE07B078105A5
:104A9000910560F447E02D813E81429FF001439FE4
:104AA000F00D1124ED5DFD4F51E011C06034AFE118
:104AB0007A078105910568F447E02D813E81429F88
:104AC000F001439FF00D1124ED5DFD4F52E0558341
:104AD0000CC027E0AD81BE812A9FF0012B9FF00D15
:104AE0001124ED5DFD4F33E03583A7E04D815E81FC
:104AF000A49FF001A59FF00D1124ED5DFD4F2581D0
:104B0000022E04C096958795779567950A94D2F7FB
:104B100049815A8102C0440F551F2A95E2F75183FB
:104B200040836115710551E08507910568F427E020
:104B3000AD81BE812A9FF0012B9FF00D1124ED5D08
:104B4000FD4F7383628304C04FEF5FEF5383428353
:104B50008091FC0580934D028F5F863019F0809321
:104B6000FC0502C01092FC05E091FF05F0910006E3
:104B7000C101D801868F978FA0A3B1A3C092AE02C6
:104B8000D092AF02E092B002F092B102A301920182
:104B9000C701B6010E94D335A50194010E942B39AB
:104BA0006093AA027093AB028093AC029093AD0223
:104BB0002091BB023091BC024091BD025091BE02D7
:104BC000B101C8010E94C9368111F4C820E030E06B
:104BD000A901B101C8010E94EB3890911E0118167D
:104BE00014F092FF04C0916090931E0119C01092BE
:104BF00000061092FF059091DA028091FB0589175B
:104C000009F4D8C881E0890F803109F480E020914F
:104C1000D802921302C08093D8028093DA02CAC8E5
:104C2000EF960FB6F894DEBF0FBECDBFDF91CF91E8
:104C30001F910F91FF90EF90DF90CF90BF90AF90BA
:104C40009F908F907F906F905F904F903F902F90AC
:104C50000895CF93DF93C091FF05D0910006209770
:104C6000C9F08091A90281608093A9026091BF027E
:104C70007091C0028091C1029091C2029B01AC016F
:104C80000E942B396A8B7B8B8C8B9D8B109200063C
:104C90001092FF05DF91CF9108952F923F924F928E
:104CA0005F926F927F928F929F92AF92BF92CF92BC
:104CB000DF92EF92FF920F931F93CF93DF93309089
:104CC000FB05311002C0D0E101C0D32DD150C091FD
:104CD000D802CD1709F416C1ED2EF12C22E3D29F94
:104CE0008001112405521D4FF801A688B788C08C99
:104CF000D18C628D738D848D958D9B01AC010E944A
:104D0000D435F801268D378D40A151A10E942B3951
:104D10004B018C019B01AC01B501C6010E94C93653
:104D200087FD02C05401680182E38E9DF0018F9DD2
:104D3000F00D1124E552FD4FC501D601828B938BF6
:104D4000A48BB58BD11101C0D0E1D150CD1307C0D8
:104D50008091DA02C81368C00E94292665C022E348
:104D60002E9DC0012F9D900D11249C0125523D4F79
:104D7000790192E3292EAD2EB12C2A9CC0012B9CE7
:104D8000900D1124FC01E552FD4F6F01D11101C0BE
:104D9000D0E1D1508091DA028D1302C00E94292601
:104DA0002A9C80012B9C100D112405521D4FF801E7
:104DB00086889788A08CB18CA5019401628973893B
:104DC000848995890E94C936882359F1F801628D3A
:104DD000738D848D958D9B01AC010E94D435F801B3
:104DE000268D378D40A151A10E942B39F7012289D0
:104DF0003389448955890E94D4352B013C019B019C
:104E0000AC01C501B4010E94EB38F80118162CF46E
:104E1000428A538A648A758A04C0828A938AA48AE1
:104E2000B58A7601CD13A7CFF2E3CF9F800111247D
:104E300005521D4FCF5FC03109F4C0E0D091D802B8
:104E400082E3282EC31509F45BC0CC2ED12C2C9CF8
:104E5000C0012D9C900D11249C0125523D4F7901DC
:104E6000F8014288538864887588F901828893889C
:104E7000A488B588A5019401C301B2010E94C93676
:104E800087FF24C0F801628D738D848D958D9B0101
:104E9000AC010E94D435F801268D378D40A151A177
:104EA0000E942B39A30192010E94D4352B013C01B1
:104EB0009B01AC01C501B4010E94EB38181634F413
:104EC000F701428A538A648A758ADC2F2C9CF00190
:104ED0002D9CF00D1124E552FD4F26893789408D18
:104EE000518D62897389848995890E94C93681119F
:104EF00001C0DC2FCF5FC03109F4C0E08701A2CF31
:104F0000D093D802DF91CF911F910F91FF90EF9036
:104F1000DF90CF90BF90AF909F908F907F906F90D9
:104F20005F904F903F902F9008952F923F924F9215
:104F30005F926F927F928F929F92AF92BF92CF9229
:104F4000DF92EF92FF920F931F93CF93DF93CDB732
:104F5000DEB7C454D1090FB6F894DEBF0FBECDBF83
:104F60003B010091FB05202E312C22E3229DA00164
:104F7000239D500D1124BA0165527D4F7AAF69AF60
:104F8000FB0111922A95E9F7F3012085FB01218BA2
:104F9000F3014481558166817781E9ADFAAD46A779
:104FA00057A760AB71AB21FF40C02CE0E1E0F1E01E
:104FB000DE01599601900D922A95E1F78BAB9CABDF
:104FC0002BE231E03EAB2DABBE01635F7F4F2396FA
:104FD0007FAF6EAF2397CE01499621969FAF8EAFDC
:104FE0002197E2E30E9FC00111249C0125523D4F01
:104FF0003EAF2DAF685E7F4F7CAF6BAF78AF6FABCE
:1050000010E082E3829D9001839D300D1124C9013F
:1050100085529D4FFC013C962596FFAFEEAF25973C
:105020002C01F0E14F0E511C3CC02CE0E1E0F6E019
:10503000BFCFEDADFEAD2193319341935193FEAFC0
:10504000EDAF2596EEADFFAD2597C080D180E28013
:10505000F380C216D306E406F50610F469017A015E
:105060002596EEADFFAD2597C082D182E282F38214
:105070000E947D37A50194010E94D336EFA9F8ADB7
:105080006193719381939193F8AFEFAB20E030E09F
:10509000A9010E94C93687FD42C01F5F133009F481
:1050A0004CC0EBA9FCA96191719181919191FCABEC
:1050B000EBABEDA9FEA981909190A190B190FEABD0
:1050C000EDABA50194010E942B390E94F83823967C
:1050D000EEADFFAD239761937193819391932396E6
:1050E000FFAFEEAF23972196EEADFFAD2197C190B4
:1050F000D190E190F1902196FFAFEEAF21976C191E
:105100007D098E099F099B01AC0197FF92CF222751
:105110003327A901261B370B480B590B8ACF1123C4
:1051200021F0113021F080E803C080E201C080E46A
:10513000F2019081892B8083B0CFCD28CE28CF2853
:1051400009F496C1CE0185960E942E314B015C0177
:1051500022E3229DC001239D900D11249C01255224
:105160003D4F7901F901868E978EA0A2B1A2BE01B2
:105170006B5D7F4F83E491E00E94D830F701628F2E
:10518000738F848F958FBE016B5D7F4F87E391E0B6
:105190000E94D830F70166A377A380A791A7118951
:1051A00010FD12C0F301208131814281538113FD32
:1051B00006C0F70122A733A744A755A709C0C50118
:1051C000B4010E942B39F70162A773A784A795A7A2
:1051D0008091DA02081711F011FF0DC082E3829D61
:1051E000F001839DF00D1124E552FD4F128A138AC0
:1051F000148A158A54C02DE036E03CAB2BAB8E01EF
:105200000F5F1F4FBE016F5C7F4F7AAB69ABC12C44
:10521000D12C76010DAB1FABEBA9FCA9819091902D
:10522000A190B190FCABEBABEBADFCAD41905190DC
:1052300061907190FCAFEBAFA3019201C501B40185
:105240000E942B399B01AC01C701B6010E94D335E6
:105250006B017C01A5019401C301B2010E94D33509
:10526000F80161937193819391938F0129A93AA9D0
:105270006BAD7CAD2617370779F62FEE3FEF4FE782
:105280005FE3C701B6010E94EB3818166CF482E3A5
:10529000829DF001839DF00D1124E552FD4F12A275
:1052A00013A214A215A271C02FEE3FEF4FE75FEBE0
:1052B000C701B6010E94C93687FF11C082E3829DF3
:1052C000F001839DF00D1124E552FD4F89E996E729
:1052D000A6E9BEE782A393A3A4A3B5A356C08DA954
:1052E0009FA90E942E316DA97FA983E491E00E94BD
:1052F000D8304B015C01A701960160E070E080E8C6
:105300009FE30E94D33520E030E040E05FE30E945D
:105310002B390E94CA396B017C01209160013091C8
:1053200061014091620150916301C501B4010E9485
:105330002B39A70196010E942B394B015C01A70173
:10534000960160E070E080E89FE30E94D3359B0106
:10535000AC01C501B4010E94D3366B017C0120E091
:1053600030E0A9010E94C93687FF03C0C12CD12CAF
:10537000760182E3829DF001839DF00D1124E552B8
:10538000FD4FC2A2D3A2E4A2F5A282E3829D8001D6
:10539000839D100D112405521D4FF801818981FD57
:1053A00069C089AD9AAD0E94351C6B017C0180906B
:1053B000190690901A06A0901B06B0901C06A50135
:1053C00094010E94EB3818162CF4A5019401C50134
:1053D000B40104C0A7019601C701B6010E942B3990
:1053E000F801668B778B808F918F82E3829D80019D
:1053F000839D100D112405521D4FF80182A093A02A
:10540000A4A0B5A0A501940166897789808D918DAE
:105410000E94EB3818162CF4F801868A978AA08E21
:10542000B18EC0921906D0921A06E0921B06F09235
:105430001C068CE0FE01B596ADE0B6E001900D9241
:105440008A95E1F78CE0FE013D96A1E0B6E001907F
:105450000D928A95E1F78091D9028093FB058F5FC9
:10546000803109F480E08093D9020E944D2602C069
:1054700080E001C081E0CC5BDF4F0FB6F894DEBF67
:105480000FBECDBFDF91CF911F910F91FF90EF9095
:10549000DF90CF90BF90AF909F908F907F906F9054
:1054A0005F904F903F902F900895CF93DF930E948D
:1054B0004C1580E3E8EAF2E0DF011D928A95E9F7F6
:1054C000CFEFD1E083E2FE0111928A95E9F71092C5
:1054D00000061092FF051092220210924D0281E008
:1054E0008093FC051092FE010E941B158091FD0126
:1054F0008F878BB1837E9091FC01892B8BB98BB107
:105500008F719091FD01892B8BB9DF91CF91089517
:10551000CF93DF93C1E1D7E08991882319F00E94EE
:105520000732FACFDF91CF910895CF93DF9321E532
:10553000829FC0011124EC01DD5F40E550E0BE0117
:1055400081E197E00E94571E892B69F410921107A0
:105550000E94F73340E550E061E177E0CE010E9420
:10556000C91C80E001C081E0DF91CF9108959FB711
:10557000F89420912006822B809320069FBF0895E7
:105580009FB7F89420911F06822B80931F069FBF20
:1055900008959FB7F89480931E069FBF08952FB774
:1055A000F89490911D068095892380931D062FBF46
:1055B00008959FB7F89420911D06822B80931D06B5
:1055C0009FBF08958F929F92AF92BF92EF92FF92EA
:1055D0000F931F93CF93DF93EC010FE411E07C0155
:1055E0008CE0E80EF11C89909990A990B99020E088
:1055F00030E0A901C501B4010E94C93687FD14C07D
:10560000F80181919191A191B1918F019C01AD011E
:105610005058C501B4010E94EB3818162CF0CE1575
:10562000DF0509F780E001C081E0DF91CF911F9194
:105630000F91FF90EF90BF90AF909F908F90089543
:105640008F929F92AF92BF92CF92DF92EF92FF9292
:105650000F931F93CF93DF93EB012BE2E22E21E018
:10566000F22E8C016B018CE0C80ED11C69917991EE
:1056700089919991F70181909190A190B1907F01CA
:105680000E947D37A50194010E94D336F8016193F1
:105690007193819391938F01CC15DD0539F7DF91DB
:1056A000CF911F910F91FF90EF90DF90CF90BF901F
:1056B000AF909F908F9008950E94F733109226012B
:1056C000089596B1892F877049F0892F8095817050
:1056D00091FF826092FD03C08460089580E0089588
:1056E0001F920F920FB60F9211242F933F934F9357
:1056F0005F936F937F938F939F93AF93BF93EF933A
:10570000FF930E94612B882391F080FF03C00E94C9
:105710005F340DC082FF04C080911D06826005C009
:1057200081FF05C080911D06886080931D06FF9152
:10573000EF91BF91AF919F918F917F916F915F9109
:105740004F913F912F910F900FBE0F901F90189582
:10575000109200019091700197FD03C090E2909328
:105760000001882331F09091000180E28927809325
:10577000000108958F929F92AF92BF92CF92DF92D5
:10578000EF92FF920F931F93CF93DF93CDB7DEB7C6
:105790002D970FB6F894DEBF0FBECDBF6B017C0115
:1057A000042F20E030E0A9010E94C93687FF07C01E
:1057B0008DE20E940732F7FAF094F7F8F094102F78
:1057C000123060F020E030E048EC52E4C701B6014E
:1057D0000E942B396B017C011250F2CF00FF0AC0EE
:1057E00020E030E040E251E4C701B6010E942B39CD
:1057F0006B017C0120E030E040E05FE3C701B601CF
:105800000E94D4350E94453710E03AE0832E912C57
:10581000A12CB12C611571058105910591F0EE2443
:10582000E394F12CEC0EFD1EE10EF11CA501940198
:105830000E94543A605DF7016083B901CA011F5F9D
:10584000E9CF80E3101748F4E1E0F0E0EC0FFD1F32
:10585000E10FF11D80831F5FF5CF101313C0FE0110
:10586000E10FF11D80E381831F5F0CC0101303C0A3
:105870008EE20E940732FE01E10FF11D80810E943D
:10588000073211501111F2CF2D960FB6F894DEBFEA
:105890000FBECDBFDF91CF911F910F91FF90EF9081
:1058A000DF90CF90BF90AF909F908F900895209100
:1058B000700120FF08C02BE832E441E25DE30E9462
:1058C0002B3941E001C040E00C94BA2B20917001CB
:1058D00020FF08C02BE832E441E25DE30E942B394F
:1058E00044E001C043E00C94BA2B0F931F93CF9375
:1058F0008C01C0E0F80161917191819191918F01CA
:105900000E94662CC23019F08CE20E940732CF5FF1
:10591000C33081F7CF911F910F910895CF93DF93FB
:10592000843630F06AE00E94343AC0E3C90F03C005
:10593000C0E08A3030F06AE00E94343AD0E3D90FF8
:1059400001C0D0E0805D0E940732DD2319F08D2F69
:105950000E940732CC2329F08C2FDF91CF910C9439
:105960000732DF91CF910895CF93DF93FC018491AB
:10597000EF012196882321F00E940732FE01F7CF24
:10598000DF91CF9108958CE093E00C94B42CCF93E9
:10599000C82F85E193E00E94B42C8C2F0E948E2C9E
:1059A000CF910C94C32C811104C08CE193E00C9432
:1059B000B42C0C94C72CCF93DF93C0E08C2F0E94A3
:1059C000952A81110EC0109211078EE30E940732B2
:1059D0000E94882A8AE30E94073287E00E94C72C2F
:1059E00012C080911107882371F00E94A501D82F61
:1059F0008EE30E9407320E94882A8AE30E940732BF
:105A00008D2F0E94D32CCF5FC230C1F6DF91CF9192
:105A10000895CF92DF92EF92FF92CF93DF93D82F2A
:105A20006A017B01C22F84E20E9407328D2F0E94FF
:105A30008E2C8DE30E9407324C2FC701B6010E94C5
:105A4000BA2BDF91CF91FF90EF90DF90CF900C9425
:105A5000C32CCF93DF93D82FC62F84E20E94073246
:105A60008D2F0E948E2C8DE30E9407328C2F0E9476
:105A70008E2CDF91CF910C94C32CEF92FF920F9359
:105A80001F93CF93DF9360915B0170E080E00E94F1
:105A9000292D60915E0170E081E00E94292D6091C6
:105AA0005C0170E082E00E94292D60915D0170E050
:105AB00083E00E94292D6091700162FB662760F9E6
:105AC00070E084E00E94292D6091700166FB6627DA
:105AD00060F970E085E00E94292D80917001082E08
:105AE000000C990B692F661F6627661F70E086E021
:105AF0000E94292D60915F0170E08AE00E94292DAB
:105B00004091600150916101609162017091630167
:105B100023E08BE00E94092D4091640150916501C2
:105B2000609166017091670123E08CE00E94092D6D
:105B300060917001617070E08DE00E94292D60918C
:105B4000700165FB662760F970E084E10E94292DF1
:105B50006091700163FB662760F970E085E10E9447
:105B6000292D609170016295617070E086E10E945C
:105B7000292D6091710170E087E10E94292D4091EB
:105B8000720150917301609174017091750123E06D
:105B900088E10E94092D4091760150917701609132
:105BA00078017091790123E089E10E94092D6091CB
:105BB0007A0170917B018AE10E94292D40917C013C
:105BC00050917D0160917E0170917F0123E08BE116
:105BD0000E94092D409168015091690160916A010C
:105BE00070916B0120E08EE10E94092D40916C01C3
:105BF00050916D0160916E0170916F0120E08FE115
:105C00000E94092D609170016695617070E080E2DC
:105C10000E94292DD4E6F12C0BE211E083E0E82E5E
:105C2000ED0ECD2F82E0F81691F0E3E0FE16E9F0DC
:105C3000F1E0FF1631F0F8014081518162817381FA
:105C40001AC0F801448555856685778514C020E023
:105C500030E041E655E4F801608D718D828D938DC1
:105C60000E94D336AB01BC0106C0F80144A155A186
:105C700066A177A1705823E08C2F0E94092D0C5F3C
:105C80001F4FCF5FEC12CECFD65FF394DC3821F6F6
:105C9000DF91CF911F910F91FF90EF9008958DE5C7
:105CA0000E9407320C94C32CCF93DF93CDB7DEB79D
:105CB0002C970FB6F894DEBF0FBECDBF8FE093E0F8
:105CC0000E94B42C6DE071E0CE0101960E94202B61
:105CD000CE0101960E94752C8AE30E9407328091C2
:105CE0001F010E948E2C0E944F2E2C960FB6F89406
:105CF000DEBF0FBECDBFDF91CF9108951F920F92EF
:105D00000FB60F9211242F933F934F935F936F938E
:105D10007F938F939F93AF93BF93EF93FF93809164
:105D20001A01813049F080911E06811105C00E9440
:105D30005F3481E00E94C92AFF91EF91BF91AF913A
:105D40009F918F917F916F915F914F913F912F9193
:105D50000F900FBE0F901F90189593B19671809180
:105D6000700186FD02C086E19827992349F091FBD6
:105D7000882780F992FD8260907119F084600895FF
:105D800080E008952F923F924F925F926F927F92A0
:105D90008F929F92AF92BF92CF92DF92EF92FF923B
:105DA0000F931F93CF93DF93CDB7DEB7A1970FB6B5
:105DB000F894DEBF0FBECDBF90911B019111BDC104
:105DC0008D8FFE013D9689E0DF011D928A95E9F7EE
:105DD00086E08D8BEBE2F1E0FA8FE98F5F019E01A7
:105DE0002A5E3F4F490100E010E0C12CD12C760122
:105DF0009D8D892F90E09C8F8B8F802F002321F029
:105E0000013021F090E103C094E001C098E0D4019A
:105E10009D934D01EB8DFC8D02C0F595E7958A951C
:105E2000E2F7E0FF1BC020E030E040EC5FEBD50183
:105E300094966D917D918D919C9197970E942B39AD
:105E4000362E472E582E692EA70196010E94C9367C
:105E500087FD04C0C32CD42CE52CF62C0F5F1F4FFC
:105E6000B4E0AB0EB11C0330110539F62090760179
:105E700030907701409078015090790194E0A92EFC
:105E8000BB24B39461E071E0CE0101960E94202B07
:105E900080917101E82FF0E0FF8FEE8FFE013196C7
:105EA00081E0682E81E0782E79A268A2CE01469624
:105EB0004C0180E090E000E010E0B701A6017058CE
:105EC0002B8D3C8D082E02C0359527950A94E2F75C
:105ED00020FF23C00F5FA8A1B9A11D921D921D92A2
:105EE0001C9213972E8D3F8D082E02C03595279555
:105EF0000A94E2F720FF03C0BB2019F007C0BB20C3
:105F000029F0C082D182E282F38204C040835183AF
:105F100062837383D4012C91122B0196BFEF8B1AED
:105F20009B0A349628A139A12C5F3F4F39A328A39F
:105F30008330910529F6602F70E080E090E00E94A8
:105F40007B370E94CA399B01AC0110932001C2012A
:105F5000B1010E942B396D877E878F87988BBE0198
:105F6000635F7F4FCE0101960E94952734E0309306
:105F70001E010E94BC1E0E94CA17BB20E9F00E94AD
:105F8000AD2EFE01769620E030E090E06191462F44
:105F9000412359F0AC01022E02C0559547950A9451
:105FA000E2F740FF02C0609516232F5F3F4F23307A
:105FB000310561F7109320010E94BC1E80911D06DF
:105FC000847339F110911D0614FF03C086E00E940E
:105FD000C92A15FF03C087E00E94C92AB11007C073
:105FE0000E94AD2E9D8D892339F088E003C012FFF9
:105FF00003C089E00E94C92A80911E06882329F0E7
:106000000E945F340E94EB3298C084E00E94CF2A45
:1060100004C0812F8C7109F0B0CF0E94552A0091E5
:106020007A0110917B010115110549F0AFE9BFE03C
:106030001197F1F700C0000001501109F4CFB1E051
:10604000BB26C9F020E030E040EA50E460917C01DA
:1060500070917D0180917E0190917F010E942B398A
:106060006B017C01209072013090730140907401AB
:106070005090750110C0C0907C01D0907D01E090DF
:106080007E01F0907F012090760130907701409062
:10609000780150907901AA94A110F4CEE09071019A
:1060A000F12C80907C0190907D01A0907E01B090B9
:1060B0007F018B8D9C8D002E02C0959587950A944B
:1060C000E2F780FF29C0C701002E02C09595879591
:1060D0000A94E2F780FD18C0E98DFA8D84A195A19C
:1060E000A6A1B7A1BC01CD019058A50194010E94C1
:1060F000D335A98DBA8D2D913D914D915C910E9422
:106100002B390E94F83803C060E070E0CB01F30146
:1061100060837183828393830F5F1F4FF4E06F0E60
:10612000711C298D3A8D2C5F3F4F3A8F298F033098
:10613000110509F0BECF10921E01A1960FB6F8947A
:10614000DEBF0FBECDBFDF91CF911F910F91FF90AA
:10615000EF90DF90CF90BF90AF909F908F907F9007
:106160006F905F904F903F902F900895EBE6F0E096
:106170008081897E8083E8E6F0E080818E7F808365
:10618000089584B1897E84B985B1866185B980918D
:10619000700183FF0BC080916B00866180936B0060
:1061A0008091680081608093680008950C94B630F7
:1061B0006F927F928F929F92AF92BF92CF92DF9217
:1061C000EF92FF920F931F93CF93DF93EB018C011C
:1061D0005B018CE0A80EB11C89E9682E96E7792E48
:1061E00026E9822E3EE7932EC990D990E990F99046
:1061F00020E030E0A901C701B6010E94C93688231A
:10620000B9F0A7019601F8016081718182819381C3
:106210000E94D3366B017C01E894F7F89301A40146
:10622000C701B6010E94EB38181614F03601470179
:106230000C5F1F4FCA15DB05B9F6B301C401DF912E
:10624000CF911F910F91FF90EF90DF90CF90BF9073
:10625000AF909F908F907F906F9008954F925F9234
:106260006F927F92AF92BF92CF92DF92EF92FF92A6
:106270000F931F93CF93DF93EC015C018CE0A80E8A
:10628000B11C8E01C12CD12C7601F80141905190A6
:10629000619071908F0120E030E0A901C301B2014B
:1062A0000E94C936882371F0A3019201C301B20193
:1062B0000E942B399B01AC01C701B6010E94D43565
:1062C0006B017C010A151B0501F7C701B6010E948D
:1062D000CA396B017C019B01AC0160E070E080E891
:1062E0009FE30E94D3362B013C01A30192016881F8
:1062F00079818A819B810E942B3969937993899353
:106300009993AC16BD0689F7C701B601DF91CF910D
:106310001F910F91FF90EF90DF90CF90BF90AF90C3
:106320007F906F905F904F9008951F93CF93DF936E
:10633000142F20E030E040EA51E40E942B390E9403
:10634000B2360E944C37EB012097D1F080911B01AF
:10635000811116C0111103C00E94EB3206C00E94C9
:10636000E21780911C0181FD0BC02FEF80E792E0C6
:10637000215080409040E1F700C000002197E4CF19
:10638000DF91CF911F910895E1E0F1E0A1E0B6E047
:1063900041915191619171914D935D936D937D9375
:1063A00081E0ED30F807A1F708950E94A81C892B21
:1063B00019F082E00C94D92A08951F920F920FB61B
:1063C0000F9211248F939F93EF93FF938091100767
:1063D000E82FF0E0E955F94F90819093C6008F5F68
:1063E000893609F480E0809310079091A6068913FE
:1063F00005C08091C1008F7D8093C100FF91EF9116
:106400009F918F910F900FBE0F901F901895E09164
:10641000A60691E09E0F993631F490E004C02091D9
:106420001D0624FD0FC0209110072917C1F3F0E0CD
:10643000E955F94F80839093A6068091C100806250
:106440008093C100089590911B01911108C08111A2
:1064500002C0439802C086FD439A10922501089518
:106460004F925F926F927F928F929F92AF92BF9264
:10647000CF92DF92EF92FF926B017C0180906C01D2
:1064800090906D01A0906E01B0906F0140906801F6
:106490005090690160906A0170906B01A3019201B4
:1064A000C501B4010E94EB3887FF08C0A70196011F
:1064B000C301B2010E94C936181654F04092270158
:1064C000509228016092290170922A0186E23CC014
:1064D000A7019601C501B4010E94EB3887FD11C0E8
:1064E00020E030E0A901C701B6010E94C9368092C0
:1064F000270190922801A0922901B0922A0187E0F9
:1065000023C0C0922701D0922801E0922901F09285
:106510002A01A5019401C701B6010E94D33520913B
:10652000A2063091A3064091A4065091A5060E94B0
:106530002B390E94B83720E030E040EE50E40E9452
:10654000D4350E944C37862FFF90EF90DF90CF908C
:10655000BF90AF909F908F907F906F905F904F9083
:1065600008958093B300811104C08091B0008F77AB
:1065700003C08091B00080688093B000089590912E
:106580001B01911127C081110FC080E090E0A0EEA7
:10659000B0E48093270190932801A0932901B09340
:1065A0002A01BC01CD0110C0803111F42D9801C029
:1065B0002D9A9091700191FF05C0803219F440E04E
:1065C00050E0BA01CB01BA010E9430320E94B132D0
:1065D000109225010895CF92DF92EF92FF921F93C0
:1065E000CF93DF930E94E21780911C01882309F466
:1065F000F6C00E94A81C009771F4C0918901809197
:106600008801C82BC0908B01D0908C01E0908D0147
:10661000F0908E0106C0FC01C189C6A4D7A4E0A8F1
:10662000F1A88091700181FF03C080E20E94B72A27
:10663000DC2FD07311E0C07480911C01882309F411
:10664000CEC090911B019111CAC080FFC5C090912E
:106650001A01292F207C09F474C082FD12C0109207
:10666000240140E050E0BA0180E00E94BF3280E0A7
:106670000E94233280911C018D7F846080931C01D5
:10668000ABC09038E1F481EF91E00E94B42C8AE530
:1066900091E00E94B42C0E944F2E40E050E0BA01DD
:1066A00080E00E94BF3280E00E9423320E944C159D
:1066B00080911B01811193C00E94E217F9CF9034A1
:1066C00019F48F7D80931C0180911C0183FF84C08D
:1066D000909189019923C1F081FD16C080917001CC
:1066E00081FF06C080911E01886080931E010CC04E
:1066F000B701A6018D2F0E94BF3241E060E070E03B
:1067000080E890E40E94953180918801882371F09F
:1067100080911C0181FD0AC08C2F0E94233241E030
:1067200060E070E080E89FE30E94953180911C0159
:1067300081FD52C0806180931C0182E00E94D92AB1
:106740004BC0809124018823C9F181FF0DC0809145
:1067500089018823B1F040E050E0BA0180E00E9456
:10676000BF321093240138C08C70B1F1809189013F
:1067700081110AC08091240183FF03C082E00E943E
:10678000D92A1092240128C081EF91E00E94B42CF4
:1067900083E691E00E94B42C0E944F2E80917001FC
:1067A00081FF06C080911E01886080931E01E2CFA8
:1067B000B701A6018D2F0E94BF32DCCF80911E0150
:1067C00083FF0AC0B701A6018D2F0E94BF328091BE
:1067D0001E01877F80931E010E94E2172DCFDF915B
:1067E000CF911F91FF90EF90DF90CF9008950E947E
:1067F000D5310E94EB3280911B01811108C00E94AB
:10680000A81C892BB1F780911A01883091F3089563
:10681000CF92DF92EF92FF92CF9390911A01923034
:1068200079F06A017B01C82F0E94F733B701A601F6
:106830008C2FCF91FF90EF90DF90CF900C94BF32D0
:10684000CF91FF90EF90DF90CF900895CF93DF939B
:10685000239AC0EBD0E083E0888387E08093B10087
:10686000259A20916C0130916D0140916E015091FB
:106870006F01609168017091690180916A01909146
:106880006B010E94D3359B01AC0160E070E088EFA2
:1068900091E40E94D3366093A2067093A30680937E
:1068A000A4069093A50688818F778883DF91CF9186
:1068B000089561E071E088E991E00C94202B8091CB
:1068C0001D0684FD1FC080E10E94D92A8091B0007E
:1068D0008F778093B000439890911A01892F8C7222
:1068E00021F480911E01867069F0943031F480911A
:1068F0001E06811105C086E001C083E00E94C92AFE
:106900000C944C1508951F920F920FB60F921124FC
:106910002F933F934F935F936F937F938F939F93A7
:10692000AF93BF93EF93FF93E091C600E13271F014
:1069300028F4E83179F40E945F3456C0EF3321F037
:10694000EE3741F482E003C081E001C088E00E949C
:10695000D92A4AC0E7FF37C08E2F90E0FC01E458E7
:10696000F109ED31F10508F03FC0E659FF4F0C94F5
:10697000763A80E2ECCF80911A0185FF35C080E441
:10698000E6CF81E00DC082E00BC084E009C088E062
:1069900007C080E105C080E203C080E401C080E858
:1069A0000E94C02A21C081E00BC082E009C084E0BF
:1069B00007C088E005C080E103C080E201C080E438
:1069C0000E94B72A11C0A091FA0181E08A0F813894
:1069D00009F480E09091FB01891731F0B0E0AF5DE0
:1069E000B94FEC938093FA01FF91EF91BF91AF9172
:1069F0009F918F917F916F915F914F913F912F91D7
:106A00000F900FBE0F901F901895CF93C82F0E9424
:106A1000B630CC2311F08C2F01C083E00E94C22E2F
:106A20000E94EB3280911B01811107C00E945934F2
:106A30000E94C431CF910C94C130CF9108958F92B0
:106A40009F92AF92BF92CF92DF92EF92FF920F93FD
:106A50001F93CF93DF937C016B01DC01CC91D0E0DD
:106A6000FE01EF5EF84F80818D3229F4EF0122960E
:106A7000818101E009C08B3219F0CE5ED84F03C08E
:106A8000EF012296818100E0912CF0E010E020E0FF
:106A900030E0A9015E01E0EDE80FEA30D0F4FF5FDD
:106AA000F93098F491101150A5E0B0E00E947C3AC2
:106AB000DC01CB01880F991FAA1FBB1F9C01AD01F0
:106AC0002E0F311D411D511D0AC0911008C01F5FBE
:106AD00006C0EE3F41F4911006C09924939421968C
:106AE000D5018C91D7CFFF2309F44FC0CA01B9015A
:106AF0000E947B374B015C0120E030E0A9010E943D
:106B0000C936882349F11F3F64F42AE037ED43E298
:106B10005CE3C501B4010E942B394B015C011E5F8F
:106B2000F2CF1F3F59F42DEC3CEC4CEC5DE3C5017A
:106B3000B4010E942B394B015C010EC0112361F09E
:106B400020E030E040E251E4C501B4010E942B395D
:106B50004B015C011150F2CF002351F0B7FAB09411
:106B6000B7F8B094F60180829182A282B38206C007
:106B7000D6018D929D92AD92BC921397C151D74090
:106B8000C150F701C08381E001C080E0DF91CF9167
:106B90001F910F91FF90EF90DF90CF90BF90AF903B
:106BA0009F908F9008955058BB27AA270E94EB35DD
:106BB0000C9485380E944C3838F00E94533820F0ED
:106BC00039F49F3F19F426F40C9422380EF4E09522
:106BD000E7FB0C94F337E92F0E94AA3858F3BA1751
:106BE000620773078407950720F079F4A6F50C94E3
:106BF000E4380EF4E0950B2EBA2FA02D0B01B9014D
:106C000090010C01CA01A0011124FF27591B99F022
:106C1000593F50F4503E68F11A16F040A22F232F2E
:106C2000342F4427585FF3CF469537952795A7957E
:106C3000F0405395C9F77EF41F16BA0B620B730B25
:106C4000840BBAF09150A1F0FF0FBB1F661F771F96
:106C5000881FC2F70EC0BA0F621F731F841F48F44B
:106C6000879577956795B795F7959E3F08F0B0CFD4
:106C70009395880F08F09927EE0F979587950895BB
:106C80000E944C3860F080E891E009F49EEF0E9489
:106C9000533828F040E851E071F45EEF0CC00C94DA
:106CA00022380C94E438E92FE0780E94AA3840F3A7
:106CB000092E052AB1F3261737074807590738F078
:106CC0000E2E07F8E02569F0E025E0640AC0EF63C6
:106CD00007F8009407FADB01B9019D01DC01CA0144
:106CE000AD01EF930E94EA360E9485380E948336F8
:106CF0005F91552339F02BED3FE049E450FD49EC1D
:106D00000C94D4350895DF93DD27B92FBF7740E881
:106D10005FE31616170648075B0718F4D92F0E9481
:106D2000F0389F938F937F936F930E940A3AEEE01F
:106D3000F1E00E9425380E9485382F913F914F91B4
:106D40005F910E943E39DD2351F09058A2EA2AED6E
:106D50003FE049EC5FE3D0785D270E94EB35DF919F
:106D60000C9485380E94CC3890F09F3748F49111EC
:106D700016F40C94E53860E070E080E89FE3089535
:106D800026F01B16611D711D811D0C94F9370C94A2
:106D900014380E94CF3708F481E008950E945C38CF
:106DA000E3950C9496380E94E7360C9485380E943F
:106DB000533858F00E944C3840F029F45F3F29F0D6
:106DC0000C94F33751110C94E5380C9422380E943E
:106DD000AA3868F39923B1F3552391F3951B550B0A
:106DE000BB27AA2762177307840738F09F5F5F4F9E
:106DF000220F331F441FAA1FA9F335D00E2E3AF0DD
:106E0000E0E832D091505040E695001CCAF72BD0F4
:106E1000FE2F29D0660F771F881FBB1F2617370745
:106E20004807AB07B0E809F0BB0B802DBF01FF2777
:106E300093585F4F3AF09E3F510578F00C94F3372A
:106E40000C94E5385F3FE4F3983ED4F3869577954C
:106E50006795B795F7959F5FC9F7880F911D969530
:106E6000879597F90895E1E0660F771F881FBB1F8C
:106E7000621773078407BA0720F0621B730B840B39
:106E8000BA0BEE1F88F7E09508950E944C3768947E
:106E9000B1110C94E53808950E94B23888F09F57DC
:106EA00098F0B92F9927B751B0F0E1F0660F771F2E
:106EB000881F991F1AF0BA95C9F714C0B13091F024
:106EC0000E94E438B1E008950C94E438672F782FDD
:106ED0008827B85F39F0B93FCCF3869577956795E9
:106EE000B395D9F73EF490958095709561957F4F55
:106EF0008F4F9F4F0895E89409C097FB3EF49095FB
:106F00008095709561957F4F8F4F9F4F9923A9F082
:106F1000F92F96E9BB279395F69587957795679511
:106F2000B795F111F8CFFAF4BB0F11F460FF1BC055
:106F30006F5F7F4F8F4F9F4F16C0882311F096E9E8
:106F400011C0772321F09EE8872F762F05C0662396
:106F500071F096E8862F70E060E02AF09A95660F4F
:106F6000771F881FDAF7880F9695879597F9089508
:106F70000E94CC3890F09F3748F4911116F00C9491
:106F8000E53860E070E080E89FEB089526F41B167A
:106F9000611D711D811D0C94F9370C941438990FE3
:106FA0000008550FAA0BE0E8FEEF16161706E807D3
:106FB000F907C0F012161306E407F50798F0621BF4
:106FC000730B840B950B39F40A2661F0232B242BC9
:106FD000252B21F408950A2609F4A140A6958FEFE8
:106FE000811D811D089597F99F6780E870E060E03A
:106FF0000895882371F4772321F09850872B762FFA
:1070000007C0662311F499270DC09051862B70E0BC
:1070100060E02AF09A95660F771F881FDAF7880FCD
:107020009695879597F908959F3F31F0915020F4F8
:10703000879577956795B795880F911D9695879554
:1070400097F908959FEF80EC0895DF93CF931F93F6
:107050000F93FF92EF92DF927B018C01689406C040
:10706000DA2EEF010E943E39FE01E894A5912591A8
:10707000359145915591A6F3EF010E94EB35FE0144
:107080009701A801DA9469F7DF90EF90FF900F91D4
:107090001F91CF91DF91089500240A9416161706C8
:1070A00018060906089500240A94121613061406F9
:1070B000050608950C9422380E94B238D8F3E8945B
:1070C000E0E0BB279F57F0F02AED3FE049EC06C017
:1070D000EE0FBB0F661F771F881F28F0B23A6207BA
:1070E0007307840728F0B25A620B730B840BE39585
:1070F0009A9572F7803830F49A95BB0F661F771F08
:10710000881FD2F790480C941638092E0394000C6F
:1071100011F4882352F0BB0F40F4BF2B11F460FF31
:1071200004C06F5F7F4F8F4F9F4F0895EF93E0FF35
:1071300007C0A2EA2AED3FE049EC5FEB0E94EB3585
:107140000E9485380F90039401FC9058EBE3F1E026
:107150000C94203A57FD9058440F551F59F05F3F4B
:1071600071F04795880F97FB991F61F09F3F79F069
:1071700087950895121613061406551FF2CF4695EB
:10718000F1DF08C0161617061806991FF1CF86956D
:1071900071056105089408950E94B238A0F0BEE719
:1071A000B91788F4BB279F3860F41616B11D672FF6
:1071B000782F8827985FF7CF869577956795B11DCB
:1071C00093959639C8F30895E894BB2766277727E7
:1071D000CB0197F908950E94CF3708F48FEF0895F7
:1071E0009B01AC0160E070E080E89FE30C94D33633
:1071F0000E94B23858F19E5760F19851A0F0E9F022
:10720000983020F5092E9927660F771F881F991F40
:107210000A94D1F712C0062E672F782F8827985F1F
:1072200011F4000C07C0993FB4F3869577956795E4
:107230009395D9F7611D711D811D3EF49095809540
:10724000709561957F4F8F4F9F4F089568940C9470
:10725000E5380C94E4380E943E390C9485380E943D
:107260004C3838F00E94533820F0952311F00C94DC
:10727000F3370C94223811240C94E5380E94AA3874
:1072800070F3959FC1F3950F50E0551F629FF00179
:10729000729FBB27F00DB11D639FAA27F00DB11D92
:1072A000AA1F649F6627B00DA11D661F829F22271B
:1072B000B00DA11D621F739FB00DA11D621F839FA2
:1072C000A00D611D221F749F3327A00D611D231F78
:1072D000849F600D211D822F762F6A2F11249F57C6
:1072E00050409AF0F1F088234AF0EE0FFF1FBB1FC9
:1072F000661F771F881F91505040A9F79E3F510588
:1073000080F00C94F3370C94E5385F3FE4F3983E3B
:10731000D4F3869577956795B795F795E7959F5F31
:10732000C1F7FE2B880F911D9695879597F90895C3
:107330000E94B238E8F09E37E8F09639B8F49E38EB
:1073400048F4672F782F8827985FF9CF869577952F
:10735000679593959539D0F3B62FB1706B0F711D6A
:10736000811D20F487957795679593950C94F9374F
:107370000C9414380C94E5389F930E945C380F905D
:1073800007FCEE5F0C94963819F416F40C9422382E
:107390000C9414380E94B238B8F39923C9F3B6F3A9
:1073A0009F57550B87FF0E94193A0024A0E640EA38
:1073B000900180585695979528F4805C660F771F4A
:1073C000881F20F026173707480730F4621B730B1D
:1073D000840B202931294A2BA69517940794202540
:1073E00031254A2758F7660F771F881F20F0261788
:1073F0003707480730F4620B730B840B200D311DE7
:10740000411DA09581F7B901842F9158880F969559
:10741000879508959B01AC010C942B390E94CC38C0
:1074200030F09F3710F40C94E5380C94F9370C9435
:10743000143891505040660F771F881FD2F7089577
:107440009F938F937F936F93FF93EF939B01AC0177
:107450000E942B39EF91FF910E9425382F913F9187
:107460004F915F910C942B39991B79E004C0991FBF
:10747000961708F0961B881F7A95C9F7809508958E
:10748000AA1BBB1B51E107C0AA1FBB1FA617B7074A
:1074900010F0A61BB70B881F991F5A95A9F7809566
:1074A0009095BC01CD010895A1E21A2EAA1BBB1B29
:1074B000FD010DC0AA1FBB1FEE1FFF1FA217B307C0
:1074C000E407F50720F0A21BB30BE40BF50B661FD6
:1074D000771F881F991F1A9469F76095709580959A
:1074E00090959B01AC01BD01CF010895EE0FFF1FE8
:1074F0000590F491E02D09940E94873AA59F900D84
:10750000B49F900DA49F800D911D11240895A29FFA
:10751000B001B39FC001A39F700D811D1124911D67
:10752000B29F700D811D1124911D0895FB01DC0196
:1075300004C08D910190801921F441505040C8F74A
:0A754000881B990B0895F894FFCF03
:00000001FF
